:100000000C942A001895000018950000189500001F
:10001000189500001895000018950000189500002C
:10002000189500001895000018950000189500001C
:10003000189500001895000018950000189500000C
:1000400018950000189500001895000018950000FC
:10005000189500008FE58DBFC0EEE8EF4E2E88E0CA
:100060008EBFD7E0F6E05F2EA89584B7082E877F75
:1000700084BF88E1992781BD91BDEEEFF7E0A0E64E
:10008000B0E088278D933197E9F766247FE37ABB48
:100090000E940F3186E886B980E487B9D09AD19A58
:1000A000D29AD39AD49AD59AD698B898B998BA9839
:1000B000BC9A8B9A8C9A8D9A8E9AC09AC19AC29A3F
:1000C0009698C49801080800000000000000000095
:1000D0000000065F060000000007030007030000A1
:1000E00000247E247E24000000242B6A12000000DD
:1000F0000063130864630000003649562050000076
:10010000000007030000000000003E410000000066
:100110000000413E0000000000083E1C3E080000B8
:100120000008083E080800000000E0600000000031
:1001300000080808080800000000606000000000D7
:10014000007C407C407C0000003E5149453E000060
:100150000000427F40000000006251494946000013
:100160000022494949360000001814127F1000008F
:10017000002F494949310000003C4A4949300000FC
:1001800000017109050300000036494949360000A5
:1001900000064949291E000000006C6C00000000A8
:1001A0000000EC6C00000000000814224100000078
:1001B000002424242424000000004122140800000C
:1001C0000002015909060000003E415D551E000075
:1001D000007E1111117E0000007F49494936000060
:1001E000003E414141220000007F4141413E00006C
:1001F000007F494949410000007F090909010000C9
:10020000003E4149497A0000007F0808087F00004D
:10021000007F402008047F0000403C14147C000054
:10022000007F081422410000007F40404040000051
:10023000007F0204027F0000007F0204087F0000AC
:10024000003E4141413E0000007F090909060000CF
:10025000007E0202027E0000007F0909196600008C
:1002600000264949493200000001017F01010000D8
:10027000003F4040403F0000001F2040201F000082
:10028000003F403C403F000000631408146300003E
:10029000000708700807000000244252522C00009A
:1002A000007C407C407C4000007C5070007C000062
:1002B000001C2020207C00000038555508000080DC
:1002C00080808080808080007C5050200000000072
:1002D00020545454780000003C4A49483000000043
:1002E0003844444428000000443C04043C400000DE
:1002F0003854545408000000385554550800000084
:100300007C040404080000007F040478000000005E
:100310007C4020107C0000007C4122117C00000009
:100320007C10284400000000403C04047C000000D5
:100330007C0810087C0000007C1010107C0000007D
:100340003844444438000000FC4444443800000071
:100350007804040478000000447844040800000095
:10036000085454542000000004047C0404000000DD
:100370003C40207C000000001C2040201C000000AD
:100380007C545454280000006C10106C00000000D5
:100390009CA0603C0000000044545454280000001D
:1003A000443478344400000000007700000000006E
:1003B0007C103844443800000201020100000000B3
:1003C0000108080000000000000000000000065FB7
:1003D00006000000000703000703000000247E243D
:1003E0007E24000000242B6A120000000063130822
:1003F00064630000003649562050000000000703E7
:100400000000000000003E41000000000000413EEE
:100410000000000000083E1C3E0800000008083EE6
:10042000080800000000E060000000000008080864
:1004300008080000000060600000000000201008B4
:1004400004020000003E5149453E00000000427F8A
:10045000400000000062514949460000002249491D
:1004600049360000001814127F100000002F49497F
:1004700049310000003C4A4949300000000171093F
:100480000503000000364949493600000006494985
:10049000291E000000006C6C000000000000EC6CE5
:1004A0000000000000081422410000000024242461
:1004B0002424000000004122140800000002015919
:1004C00009060000003E415D551E0000007E11112E
:1004D000117E0000007F494949360000003E41413D
:1004E00041220000007F4141413E0000007F494918
:1004F00049410000007F090909010000003E41490F
:10050000497A0000007F0808087F00000000417F52
:100510004100000000304040403F0000007F0814D0
:1005200022410000007F404040400000007F020464
:10053000027F0000007F0204087F0000003E41416E
:10054000413E0000007F090909060000003E4151BC
:10055000215E0000007F0909196600000026494954
:10056000493200000001017F01010000003F4040CE
:10057000403F0000001F2040201F0000003F403C83
:10058000403F000000631408146300000007087077
:1005900008070000007149454300000000007F414A
:1005A000410000000002040810200000000041414A
:1005B0007F000000000402010204000080808080AF
:1005C0008080808000000307000000000020545459
:1005D00054780000007F444444380000003844440C
:1005E0004428000000384444447F0000003854543C
:1005F0005408000000087E09090000000018A4A4A7
:10060000A47C0000007F0404780000000000007D4E
:1006100040000000004080847D000000007F102822
:10062000440000000000007F40000000007C04182F
:1006300004780000007C0404780000000038444482
:100640004438000000FC444444380000003844446E
:1006500044FC00000044784404080000000854549E
:100660005420000000043E4424000000003C4020D0
:100670007C000000001C2040201C0000003C60307A
:10068000603C0000006C10106C000000009CA0603A
:100690003C000000006454544C00000000083E413F
:1006A0004100000000000077000000000000414110
:1006B0003E0800000002010201000000003C262369
:1006C000263C0000E0ECF3E0A0E6B0E0ED93FC9304
:1006D00080E092E2A4E7B0E08D939C935A924A9214
:1006E000A4E7B0E08D919C91D2018D939C9382E020
:1006F0000E9460320E949F21229682E00E94532F26
:10070000A6E0B1E0E0E0F1E70E949132ACE0B1E0B8
:10071000E6E0F1E70E949132A2E1B1E0ECE0F1E71E
:100720000E949132A8E1B1E0E2E1F1E70E9491324A
:10073000AEE1B1E0E8E1F1E70E949132A4E2B1E07C
:10074000EEE1F1E70E949132A6E0B4E0E4E9F0E7DF
:100750000E945535AAE0B4E0E8E9F0E70E9455357B
:10076000AEE0B4E0ECE9F0E70E945535A2E1B4E078
:10077000E0EAF0E70E945535A6E1B4E0E4EAF0E7EC
:100780000E94553582E08093260483E080932B01FC
:10079000AAE7B0E0E8EAF0E70E945535EAE7F0E0C2
:1007A0000E94BC32A2E9B0E0EDE0FF270E943F3694
:1007B00085E0809396004091960001E0041718F0C0
:1007C00011F00C941104A6E9B0E0AD90BB24AEE7A3
:1007D000B0E0AA0CBB1CAA0CBB1CAA0DBB1D0D9142
:1007E0001D912D913C914AE050E060E070E00E9444
:1007F000C02FA6E9B0E0AD90BB24AAE7B0E0AA0CF8
:10080000BB1CAA0CBB1CAA0DBB1D4D935D936D9325
:100810007D938091960081508093960010F00C9407
:10082000DB03A7E9B0E0E0E0F1E70E949132ADE937
:10083000B0E0E6E0F1E70E949132A3EAB0E0ECE03C
:10084000F1E70E949132A9EAB0E0E2E1F1E70E940B
:100850009132AFEAB0E0E8E1F1E70E949132A5EB16
:10086000B0E0EEE1F1E70E94913281E08093BB00BD
:1008700002E310E020E030E0A2E9B0E04D915D91AC
:100880006D917C910E946E32ACEBB0E00D931D93A4
:100890002D933D93A2E8B0E00D911D912D913C91D7
:1008A000A0ECB0E00D931D932D933C937091E80064
:1008B00070687093E80082E08093E900A2E9B0E0FC
:1008C0000D911D912D913C91ACE6B0E00D931D93DF
:1008D0002D933C930E947C3182E08093620081E002
:1008E00080936300882780936400E4E2F1E70E942C
:1008F000AD2F83E08093620081E0809363008827BE
:1009000080936400E6E3F1E70E94AD2F84E08093DA
:10091000620081E080936300882780936400E8E4AC
:10092000F1E70E94AD2F85E08093620081E0809323
:100930006300882780936400EAE5F1E70E94AD2F09
:1009400086E08093620081E0809363008827809333
:100950006400ECE6F1E70E94AD2F87E0809362002F
:1009600081E080936300882780936400EEE7F1E7DD
:100970000E94AD2FE4ECF0E0A0E6B0E0ED93FC9334
:10098000E2E0F0E00E94B42F0E947C3106B347E021
:100990000423A5E6B0E00C9300916500053011F04A
:1009A0000C942205A2E9B0E00D911D912D913C918E
:1009B000A4ECB0E00D931D932D933C93A2E9B0E01D
:1009C0000D911D912D913C91A8ECB0E00D931D93DC
:1009D0002D933C930EE110E020E030E0A2E9B0E07E
:1009E0004D915D916D917C910E946E32ACECB0E0C6
:1009F0000D931D932D933D93A6E8B0E00D911D91AD
:100A00002D913C91A0EDB0E00D931D932D933C935F
:100A1000A4EDB0E0ECEAF0E70E945535A8EDB0E0B7
:100A2000ECEAF0E70E945535AAE1B4E0ECE9F0E722
:100A30000E945535AEE1B4E0E0EAF0E70E9455359A
:100A40000C945A05E0E0F0E0A4ECB0E094E00E94E1
:100A50005F36E4E0F0E0A8ECB0E094E00E945F369E
:100A6000E8E0F0E0ACECB0E094E00E945F36ECE04F
:100A7000F0E0A0EDB0E094E00E945F36E0E1F0E04D
:100A8000A4EDB0E094E00E945F36E4E1F0E0A8ED70
:100A9000B0E094E00E945F36AAE1B4E0E4E2F0E066
:100AA00094E00E945F36AEE1B4E0E8E2F0E094E06A
:100AB0000E945F3600916500053011F00C947505B9
:100AC00085E08093620081E08093630088278093B3
:100AD0006400E0E9F1E70E94AD2F06B347E004238C
:100AE000A5E6B0E00C930C945A050E947C318AEF85
:100AF00090E00E941D30379AECE2F0E0A0E4B4E010
:100B00000E945E368BE080932A0181E080934F0142
:100B1000AAE2B1E0BA93AA930E94FA22229606B3FF
:100B200047E00423A5E6B0E00C9300916500043093
:100B300011F00C94B8050E944B2FAAE2B1E08C9101
:100B40008F5F8C9300912A01053110F40C94AB0552
:100B500085E180932A010E947C31AAE2B1E0BA9338
:100B6000AA930E94FA2222968AEF90E00E941D30FA
:100B700000916500063011F00C94DC050E944B2FAB
:100B800080912A01815080932A0100912A010B3023
:100B900018F011F00C94CF058BE080932A010E948D
:100BA0007C31AAE2B1E0BA93AA930E94FA2222967B
:100BB0008AEF90E00E941D3000916500013011F035
:100BC0000C94F6050E944B2FAAE2B1E0BA93AA93C7
:100BD0000E9415292296AAE2B1E0BA93AA930E9434
:100BE000FA2222968AEF90E00E941D300091650063
:100BF000033011F00C9410060E944B2FAAE2B1E0D2
:100C0000BA93AA930E94402B2296AAE2B1E0BA932B
:100C1000AA930E94FA2222968AEF90E00E941D3049
:100C200000912A01053111F00C946F0606B347E0DC
:100C30000423A5E6B0E00C9300916500053011F0A7
:100C40000C9424060C9426060C941606E0E0F0E0C2
:100C5000A4ECB0E094E07BE70E944E36E4E0F0E0E4
:100C6000A8ECB0E094E07BE70E944E36E8E0F0E0CC
:100C7000ACECB0E094E07BE70E944E36ECE0F0E0B4
:100C8000A0EDB0E094E07BE70E944E36E0E1F0E0BA
:100C9000A4EDB0E094E07BE70E944E36E4E1F0E0A2
:100CA000A8EDB0E094E07BE70E944E36E4E2F0E08D
:100CB000AAE1B4E094E07BE70E944E36E8E2F0E07F
:100CC000AEE1B4E094E07BE70E944E368BE0809387
:100CD0002A018AEF90E00E941D300C948205009159
:100CE0002A010B3011F00C94ED2006B347E00423E9
:100CF000A5E6B0E00C9300916500053011F00C946E
:100D0000ED200E944B2F8AEF90E00E941D30E4EC12
:100D1000F0E0A0E6B0E0ED93FC930E947C3181E02E
:100D20008093620081E08093630081E0809364009F
:100D3000E4E9F1E70E94AD2F82E08093620081E058
:100D400080936300882780936400E2EAF1E70E94C1
:100D5000AD2F83E08093620081E080936300882759
:100D600080936400E4EBF1E70E94AD2F84E0809370
:100D7000620081E080936300882780936400E2EC46
:100D8000F1E70E94AD2F85E08093620081E08093BF
:100D90006300882780936400EEECF1E70E94AD2F9A
:100DA00086E08093620081E08093630088278093CF
:100DB0006400EEEDF1E70E94AD2F87E080936200C2
:100DC00081E080936300882780936400EAEEF1E776
:100DD0000E94AD2F88E08093620081E080936300E1
:100DE000882780936400EAEFF1E70E94AD2F06B3F5
:100DF00047E00423A5E6B0E00C93009165000630BF
:100E000011F00C9418070E944B2F80914F018150D4
:100E100080934F017091E80070647093E800009136
:100E20004F01013010F00C94180788E080934F01B7
:100E300000916500043011F00C9436070E944B2F8E
:100E4000AFE4B1E08C918F5F8C937091E800706497
:100E50007093E80000914F01083018F011F00C94E5
:100E600033070C94360781E080934F01A8EEB0E081
:100E70008C9186FB16F00C94B80A0E947C3100918C
:100E80004F01013011F00C94AF0781E080936200B4
:100E900081E08093630081E080936400E4E9F1E7FE
:100EA0000E94AD2F82E08093620081E08093630016
:100EB000882780936400E2EAF1E70E94AD2F83E087
:100EC0008093620081E080936300882780936400B0
:100ED000E4EBF1E70E94AD2F84E08093620081E0B3
:100EE00080936300882780936400E2ECF1E70E941E
:100EF000AD2F85E08093620081E0809363008827B6
:100F000080936400EEECF1E70E94AD2F86E08093C1
:100F1000620081E080936300882780936400EEED97
:100F2000F1E70E94AD2F87E08093620081E080931B
:100F30006300882780936400EAEEF1E70E94AD2FFA
:100F400088E08093620081E080936300882780932B
:100F50006400EAEFF1E70E94AD2F0C94AF0A023073
:100F600011F00C941D0881E08093620081E0809371
:100F70006300882780936400E4E9F1E70E94AD2FC5
:100F800082E08093620081E08093630081E080933F
:100F90006400E2EAF1E70E94AD2F83E080936200F3
:100FA00081E080936300882780936400E4EBF1E79D
:100FB0000E94AD2F84E08093620081E08093630003
:100FC000882780936400E2ECF1E70E94AD2F85E072
:100FD0008093620081E0809363008827809364009F
:100FE000EEECF1E70E94AD2F86E08093620081E095
:100FF00080936300882780936400EEEDF1E70E9400
:10100000AD2F87E08093620081E0809363008827A2
:1010100080936400EAEEF1E70E94AD2F88E08093B0
:10102000620081E080936300882780936400EAEF88
:10103000F1E70E94AD2F0C94AF0A033011F00C942D
:101040008B0881E08093620081E0809363008827B1
:1010500080936400E4E9F1E70E94AD2F82E0809381
:10106000620081E080936300882780936400E2EA55
:10107000F1E70E94AD2F83E08093620081E08093CE
:10108000630081E080936400E4EBF1E70E94AD2F00
:1010900084E08093620081E08093630088278093DE
:1010A0006400E2ECF1E70E94AD2F85E080936200DE
:1010B00081E080936300882780936400EEECF1E781
:1010C0000E94AD2F86E08093620081E080936300F0
:1010D000882780936400EEEDF1E70E94AD2F87E052
:1010E0008093620081E0809363008827809364008E
:1010F000EAEEF1E70E94AD2F88E08093620081E084
:1011000080936300882780936400EAEFF1E70E94F0
:10111000AD2F0C94AF0A043011F00C94F90881E063
:101120008093620081E0809363008827809364004D
:10113000E4E9F1E70E94AD2F82E08093620081E054
:1011400080936300882780936400E2EAF1E70E94BD
:10115000AD2F83E08093620081E080936300882755
:1011600080936400E4EBF1E70E94AD2F84E080936C
:10117000620081E08093630081E080936400E2EC90
:10118000F1E70E94AD2F85E08093620081E08093BB
:101190006300882780936400EEECF1E70E94AD2F96
:1011A00086E08093620081E08093630088278093CB
:1011B0006400EEEDF1E70E94AD2F87E080936200BE
:1011C00081E080936300882780936400EAEEF1E772
:1011D0000E94AD2F88E08093620081E080936300DD
:1011E000882780936400EAEFF1E70E94AD2F0C940A
:1011F000AF0A053011F00C94670981E0809362001A
:1012000081E080936300882780936400E4E9F1E73C
:101210000E94AD2F82E08093620081E080936300A2
:10122000882780936400E2EAF1E70E94AD2F83E013
:101230008093620081E0809363008827809364003C
:10124000E4EBF1E70E94AD2F84E08093620081E03F
:1012500080936300882780936400E2ECF1E70E94AA
:10126000AD2F85E08093620081E08093630081E090
:1012700080936400EEECF1E70E94AD2F86E080934E
:10128000620081E080936300882780936400EEED24
:10129000F1E70E94AD2F87E08093620081E08093A8
:1012A0006300882780936400EAEEF1E70E94AD2F87
:1012B00088E08093620081E08093630088278093B8
:1012C0006400EAEFF1E70E94AD2F0C94AF0A0630FC
:1012D00011F00C94D50981E08093620081E0809345
:1012E0006300882780936400E4E9F1E70E94AD2F52
:1012F00082E08093620081E080936300882780937E
:101300006400E2EAF1E70E94AD2F83E0809362007F
:1013100081E080936300882780936400E4EBF1E729
:101320000E94AD2F84E08093620081E0809363008F
:10133000882780936400E2ECF1E70E94AD2F85E0FE
:101340008093620081E0809363008827809364002B
:10135000EEECF1E70E94AD2F86E08093620081E021
:101360008093630081E080936400EEEDF1E70E94DA
:10137000AD2F87E08093620081E08093630088272F
:1013800080936400EAEEF1E70E94AD2F88E080933D
:10139000620081E080936300882780936400EAEF15
:1013A000F1E70E94AD2F0C94AF0A073011F00C94B6
:1013B000430A81E08093620081E080936300882784
:1013C00080936400E4E9F1E70E94AD2F82E080930E
:1013D000620081E080936300882780936400E2EAE2
:1013E000F1E70E94AD2F83E08093620081E080935B
:1013F0006300882780936400E4EBF1E70E94AD2F3F
:1014000084E08093620081E080936300882780936A
:101410006400E2ECF1E70E94AD2F85E0809362006A
:1014200081E080936300882780936400EEECF1E70D
:101430000E94AD2F86E08093620081E0809363007C
:10144000882780936400EEEDF1E70E94AD2F87E0DE
:101450008093620081E08093630081E08093640068
:10146000EAEEF1E70E94AD2F88E08093620081E010
:1014700080936300882780936400EAEFF1E70E947D
:10148000AD2F0C94AF0A083011F00C94AF0A81E034
:101490008093620081E080936300882780936400DA
:1014A000E4E9F1E70E94AD2F82E08093620081E0E1
:1014B00080936300882780936400E2EAF1E70E944A
:1014C000AD2F83E08093620081E0809363008827E2
:1014D00080936400E4EBF1E70E94AD2F84E08093F9
:1014E000620081E080936300882780936400E2ECCF
:1014F000F1E70E94AD2F85E08093620081E0809348
:101500006300882780936400EEECF1E70E94AD2F22
:1015100086E08093620081E0809363008827809357
:101520006400EEEDF1E70E94AD2F87E0809362004A
:1015300081E080936300882780936400EAEEF1E7FE
:101540000E94AD2F88E08093620081E08093630069
:1015500081E080936400EAEFF1E70E94AD2F8AEF0B
:1015600090E00E941D307091E8007F7B7093E8004E
:1015700000916500053011F00C94C60A0E944B2FB3
:101580008AEF90E00E941D300C94C80A0C94F70674
:101590008AEF90E00E941D3000914F01053011F05C
:1015A0000C94D40A0C94A81400914F01083011F047
:1015B0000C94DC0A0C9482050E947C3100914F014E
:1015C000043011F00C94E60A0C94A81400914F0119
:1015D000023018F011F00C94EF0A0C94A814E4EC0B
:1015E000F0E0A0E6B0E0ED93FC9300914F010230F3
:1015F00011F00C94240B81E08093620081E08093D1
:101600006300882780936400E2E0F2E70E94AD2F38
:1016100083E08093620081E0809363008827809359
:101620006400E4E1F2E70E94AD2F85E08093620060
:1016300081E080936300882780936400E6E2F2E70C
:101640000E94AD2F0C940E12033011F00C94751102
:1016500081E08093620081E080936300882780931B
:101660006400E8E3F2E70E94AD2F82E0809362001D
:1016700081E080936300882780936400EAE4F2E7C6
:101680000E94AD2F7091E80070617093E80087E0D0
:101690008093620081E08093630081E08093640026
:1016A000ECE5F2E70E94AD2F88E08093620081E0D4
:1016B00080936300882780936400EEE6F2E70E943F
:1016C000AD2F06B347E00423A5E6B0E00C930091EC
:1016D0006500053011F00C946F0B0C94D70B009142
:1016E0006500043081E008F480E08F93009165008C
:1016F000063081E010F009F080E09F918923882373
:1017000011F40C94D50BA8EEB0E08C9184FB8827E3
:1017100080F9809580FBA8EEB0E08C9184F98C93E1
:10172000A8EEB0E08C9184FB16F00C94B70B87E028
:101730008093620081E08093630081E08093640085
:10174000ECE5F2E70E94AD2F88E08093620081E033
:1017500080936300882780936400EEE6F2E70E949E
:10176000AD2F8AEF90E00E941D300C94D50B87E0DE
:101770008093620081E080936300882780936400F7
:10178000ECE5F2E70E94AD2F88E08093620081E0F3
:101790008093630081E080936400EEE6F2E70E94AC
:1017A000AD2F8AEF90E00E941D300C94610B8AEF00
:1017B00090E00E941D30A8EEB0E08C9184FB16F4FE
:1017C0000C94640D969A8AEF90E00E941D300E945E
:1017D0007C3181E08093620081E080936300882700
:1017E00080936400E0E8F2E70E94AD2F82E08093EE
:1017F000620081E080936300882780936400E2E9BF
:10180000F2E70E94AD2F83E08093620081E0809335
:101810006300882780936400E6E2F2E70E94AD2F20
:1018200006B347E00423A5E6B0E00C930091650001
:10183000053011F00C941E0C0C94200C0C94100C20
:1018400007B1007E066007B90E949732ABE3B4E0AF
:101850008D939C93EEE2F0E0ABE3B4E07BE70E9473
:101860004D36ECE2F0E0A0E4B4E00E945E368AEF90
:1018700090E00E941D30E2E9F0E00E94FA320E94FE
:101880001E330E945533E0EBF0E70E9459340E946A
:10189000C633EDE0F0E0AEEFB0E00E943F36969840
:1018A0000E9472228AEF90E00E941D300E947C31DB
:1018B00081E08093620081E08093630088278093B9
:1018C0006400E4EAF2E70E94AD2F82E080936200B8
:1018D00081E080936300882780936400E2E9F2E767
:1018E0000E94AD2F83E08093620081E080936300CB
:1018F000882780936400E6EBF2E70E94AD2F84E036
:101900008093620081E08093630088278093640065
:10191000E8ECF2E70E94AD2F85E08093620081E061
:1019200080936300882780936400EAEDF2E70E94C9
:10193000AD2F82E390E0A0E4B4E08D939C9388E027
:101940008093620081E08093630088278093640025
:10195000ECEEF2E70E94AD2FA0EEB6E0E0E4F4E09A
:101960000E94E1350E94A52F06B347E00423A5E6B7
:10197000B0E00C9300916500033011F00C94FC0C66
:10198000A0E4B4E00E945E2FA0E4B4E00D911C91AD
:10199000013050E0150710F00C94D40C81E090E079
:1019A000A0E4B4E08D939C9388E08093620081E092
:1019B00080936300882780936400E8EFF2E70E9439
:1019C000AD2F88E08093620081E0809363008827D8
:1019D00080936400ECEEF2E70E94AD2FA0EEB6E03B
:1019E000E0E4F4E00E94E1350E94A52F86E990E052
:1019F0000E941D300C943D0D013011F00C943D0DF2
:101A0000A0E4B4E00E94572FA0E4B4E00D911C9133
:101A1000043F51E0150718F011F00C94110D0C94CF
:101A2000170D84EF91E0A0E4B4E08D939C9388E0DF
:101A30008093620081E08093630088278093640034
:101A4000E8EFF2E70E94AD2F88E08093620081E02A
:101A500080936300882780936400ECEEF2E70E9495
:101A6000AD2FA0EEB6E0E0E4F4E00E94E1350E9484
:101A7000A52F86E990E00E941D3000916500053099
:101A800011F00C94620DECE2F0E0A0E4B4E07BE72E
:101A90000E944D36969807B1007E066007B90E94F5
:101AA0009732ABE2B4E08D939C93E0E3F0E0ABE2DD
:101AB000B4E07BE70E944D368AEF90E00E941D3033
:101AC0000C94640D0C94B40CE2E9F0E00E94FA323C
:101AD0000E941E330E945533E0EBF0E70E94593418
:101AE0000E94C633EDE0F0E0AEEFB0E00E943F367A
:101AF00096980E9472228AEF90E00E941D300E9408
:101B00007C31E0ECF3E0A0E6B0E0ED93FC93EEE294
:101B1000F0E0ABE3B4E00E945E36ECE2F0E0A0E47B
:101B2000B4E00E945E36E0E3F0E0ABE2B4E00E9495
:101B30005E36EBE2F4E0D190E080FF2400270E94C3
:101B40001E330E945533E4EBF0E70E9459340E94A3
:101B5000C633EDE0F0E0AEEFB3E00E943F36EBE2DB
:101B6000F4E0D190E080FF2400270E941E330E9401
:101B700055332F933F934F935F93EBE3F4E0D19072
:101B8000E080FF2400270E941E335F914F913F9118
:101B90002F910E94F833EDE0F0E0A2E0B4E00E9463
:101BA0003F36E4EBF0E70E946234E2E0F4E00E94AA
:101BB000FA320E94C633EDE0F0E0A2E0B4E00E9409
:101BC0003F36ECE9F0E70E946234E2E0F4E00E9484
:101BD000FA320E947033EDE0F0E0A2E0B4E00E943F
:101BE0003F36A8E6B0E0ECE9F0E70E945535E8E6BC
:101BF000F0E0A2E0B4E00E94EA37EDE0F0E0A2E01D
:101C0000B4E00E943F36E0E4F4E0D190E080FF24AD
:101C100000270E941E330E945533E2E0F4E00E9448
:101C2000FA320E94C633EDE0F0E0A2E0B4E00E9498
:101C30003F36E4EAF0E70E946234E2E0F4E00E941A
:101C4000FA320E94C633EDE0F0E0A2E0B4E00E9478
:101C50003F36A0EEB6E0AF93BF93E2E0F4E00E941F
:101C6000FA320E942C3011E001E0BF91AF910E9446
:101C70007C35E0EEF6E0ABE3B1E00E943A3687E077
:101C80008093620081E080936300882780936400E2
:101C9000EAE0F3E70E94AD2FABE3B1E00E94A72F8B
:101CA000E6E1F3E70E94AD2FEBE2F4E0D190E080B3
:101CB000FF2400270E941E330E945533E8EBF0E713
:101CC0000E9459340E94F833EDE0F0E0A2E0B4E065
:101CD0000E943F36E4EBF0E70E946234E2E0F4E079
:101CE0000E94FA320E94C633EDE0F0E0A2E0B4E0D8
:101CF0000E943F36ECE9F0E70E946234E2E0F4E053
:101D00000E94FA320E947033EDE0F0E0A2E0B4E00D
:101D10000E943F36E8E6F0E0A2E0B4E00E94EA3735
:101D2000EDE0F0E0A2E0B4E00E943F36E0E4F4E051
:101D3000D190E080FF2400270E941E330E9455337B
:101D4000E2E0F4E00E94FA320E94C633EDE0F0E0F7
:101D5000A2E0B4E00E943F36E4EAF0E70E94623479
:101D6000E2E0F4E00E94FA320E947033EDE0F0E02D
:101D7000A2E0B4E00E943F36A0EEB6E0AF93BF937E
:101D8000E2E0F4E00E94FA320E942C3011E001E01F
:101D9000BF91AF910E947C35E0EEF6E0ABE3B1E09D
:101DA0000E943A3681E08093620081E08093630074
:101DB000882780936400EAE0F3E70E94AD2FABE34D
:101DC000B1E00E94A72FEAE1F3E70E94AD2F80E087
:101DD0008A9380E08A9380E58A9380E08A9381E009
:101DE0008A930E94013280E08A9387E38A9380E598
:101DF0008A9387E38A9381E08A930E9401328EE47A
:101E00008A9387E38A938EE48A9380E08A9381E0C1
:101E10008A930E940132EBE3F4E0D190E080FF244A
:101E200000270E941E330E945533E8EBF0E70E9422
:101E300059340E94F833EDE0F0E0A2E0B4E00E94F3
:101E40003F36ECEBF0E70E946234E2E0F4E00E94FF
:101E5000FA320E947033EDE0F0E0A2E0B4E00E94BC
:101E60003F3687E380933E0480E08093500106B3C1
:101E700047E00423A5E6B0E00C930091650005302F
:101E800011F00C94490F8AEF90E00E941D300C94E1
:101E9000820585E090E00E941D3007B1007E06605B
:101EA00007B90E949732ABE2B4E08D939C93E4EBC8
:101EB000F0E70E946234EBE2F4E0D190E080FF248E
:101EC00000270E941E330E94C633EDE0F0E0AAE72F
:101ED000B0E00E943F36ABE3B4E04D915C91ABE2E1
:101EE000B4E00D911C910417150710F00C94800FAD
:101EF000ABE3B4E08D919C91ABE2B4E08D939C9305
:101F0000ABE2B4E00D911C91ABE3B4E04D915C9178
:101F1000041B150BABE2B4E00D931C93E2E0F4E07C
:101F20000E94FF32EBE2F4E0D190E080FF24002732
:101F30000E941E330E947033EDE0F0E0ADE2B4E0A9
:101F40000E943F36EDE2F4E00E943737EDE0F0E02A
:101F50000E94BC32ADE3B4E0DC9280913D048093FA
:101F60003F0406E340913D04041BADE3B4E00C9351
:101F700040913D0400913E04041711F40C94141098
:101F800040913E0400913D04041710F00C94EF0FB3
:101F900080913E04809396004091960000913D040C
:101FA000041718F011F00C94ED0F80E18A93A6E964
:101FB000B0E08C918A938EE38A93A6E9B0E08C918D
:101FC0008A9381E08A930E94013280919600815029
:101FD0008093960010F00C94CC0F0C941410809108
:101FE0003E048093960040913D04009196000417B2
:101FF00018F011F00C94141080E18A93A6E9B0E077
:102000008C918A938EE38A93A6E9B0E08C918A93AF
:1020100080E08A930E940132A6E9B0E08C918F5F44
:102020008C9310F40C94F30F80913D0480933E0444
:10203000EEEFF3E00E94FF32EAE7F0E00E94FA32AE
:102040000E94F833EDE0F0E0AAE7B0E00E943F36EE
:10205000ECE9F0E70E946234EAE7F0E00E94FA322D
:102060000E947033EDE0F0E0AAE7B0E00E943F3656
:10207000A8E6B0E0ECE9F0E70E945535E8E6F0E0CC
:10208000AAE7B0E00E94EA37EDE0F0E0AAE7B0E0AE
:102090000E943F36EAE7F0E00E94FF32E0E4F4E01D
:1020A000D190E080FF2400270E941E330E94C63397
:1020B000EDE0F0E0AAE7B0E00E943F368AE090E071
:1020C0000E941D30009150010D3211F00C946611E8
:1020D00080E08093500188E08093620081E08093EB
:1020E0006300882780936400E8EFF2E70E94AD2F39
:1020F000EAE7F0E00E943D38EDE0F0E0A8E6B0E06D
:102100000E943F36E8E6F0E00E94FF32ECE9F0E79B
:102110000E9459340E94C633EDE0F0E0A8E6B0E03A
:102120000E943F36A0EEB6E0AF93BF93E8E6F0E042
:102130000E94FA320E942C3011E001E0BF91AF9171
:102140000E947C35E0EEF6E0A4E3B1E00E943A366E
:10215000EAE7F0E00E94FA32E4EAF0E70E94623433
:102160000E946B3410F00C942711EAE7F0E00E9413
:10217000FA32E8E9F0E70E9462340E946B3418F00A
:1021800011F00C94C5100C94F610A0EEB6E0AF93CD
:10219000BF93EAE7F0E00E94FA320E942C3011E08F
:1021A00001E0BF91AF910E947C35E0EEF6E0ABE339
:1021B000B1E00E943A3688E08093620081E080932B
:1021C0006300882780936400ABE3B1E00E94A72FEF
:1021D000EEE1F3E70E94AD2FA4E3B1E00E94A72F48
:1021E000E2E2F3E70E94AD2F0C942511A0EEB6E0D9
:1021F000AF93BF93EAE7F0E00E94FA320E942C30DE
:1022000011E003E0BF91AF910E947C35E0EEF6E073
:10221000ABE3B1E00E943A3688E08093620081E04F
:1022200080936300882780936400ABE3B1E00E9451
:10223000A72FEEE1F3E70E94AD2FA4E3B1E00E94E7
:10224000A72FE2E2F3E70E94AD2F0C946611E4EAB7
:10225000F0E70E946234EAE7F0E00E94FA320E945E
:102260007033EDE0F0E0AAE7B0E00E943F36A0EE68
:10227000B6E0AF93BF93EAE7F0E00E94FA320E9423
:102280002C3011E001E0BF91AF910E947C35E0EE6F
:10229000F6E0ABE3B1E00E943A3688E0809362005A
:1022A00081E080936300882780936400ABE3B1E012
:1022B0000E94A72FEAE1F3E70E94AD2FA4E3B1E06B
:1022C0000E94A72FE2E2F3E70E94AD2FA0E5B1E064
:1022D0008C918F5F8C930C94370FE4ECF0E0A0E6C8
:1022E000B0E0ED93FC930C940E12063011F00C94B8
:1022F000A21181E08093620081E0809363008827CF
:1023000080936400E2E0F2E70E94AD2F83E08093C7
:10231000620081E080936300882780936400E4E199
:10232000F2E70E94AD2F85E08093620081E0809308
:102330006300882780936400E6E2F2E70E94AD2FF5
:102340000C940E12073011F00C940E1281E0809361
:10235000620081E080936300882780936400E6E256
:10236000F3E70E94AD2F82E08093620081E08093CA
:102370006300882780936400E8E3F3E70E94AD2FB1
:1023800083E08093620081E08093630088278093DC
:102390006400EAE4F3E70E94AD2F84E080936200DA
:1023A00081E080936300882780936400ECE5F3E785
:1023B0000E94AD2F85E08093620081E080936300EE
:1023C000882780936400EEE6F3E70E94AD2F86E055
:1023D0008093620081E0809363008827809364008B
:1023E000E0E8F3E70E94AD2F87E08093620081E090
:1023F00080936300882780936400E2E9F3E70E94FA
:10240000AD2F88E08093620081E08093630088278D
:1024100080936400E4EAF3E70E94AD2F06B347E03F
:102420000423A5E6B0E00C9300916500053011F09F
:102430000C941C120C9420120E944B2F0C940E1220
:102440000E94EF2080E080935001009150010F37EF
:1024500018F011F00C94531280E3809396000091D1
:1024600096000A3318F011F00C944712A0E5B1E081
:102470004C91A6E9B0E05C9191E00E94DA31A6E9C6
:10248000B0E08C918F5F8C9310F40C942F128AE043
:1024900090E00E941D30A0E5B1E08C918F5F8C939D
:1024A00010F40C942512A3E5B2E0E0E8F0E00E94FD
:1024B0008E36A8EDB3E00D931C930E947C31009101
:1024C0004F01023011F00C949B1281E08093620066
:1024D00081E080936300882780936400E6EBF3E754
:1024E0000E94AD2F83E08093620081E080936300BF
:1024F000882780936400E8ECF3E70E94AD2F84E026
:102500008093620081E08093630088278093640059
:10251000EAEDF3E70E94AD2F86E08093620081E050
:1025200080936300882780936400E6E2F2E70E94CC
:10253000AD2F0C940D13063011F00C94D51281E0E0
:102540008093620081E08093630088278093640019
:10255000E2E0F2E70E94AD2F83E08093620081E029
:1025600080936300882780936400ECEEF3E70E9479
:10257000AD2F84E08093620081E080936300882720
:1025800080936400EEEFF3E70E94AD2F86E0809326
:10259000620081E080936300882780936400E6E214
:1025A000F2E70E94AD2F0C940D13073011F00C943C
:1025B0000D1381E08093620081E08093630088279F
:1025C00080936400E6E2F3E70E94AD2F83E08093FE
:1025D000620081E080936300882780936400E0E1DB
:1025E000F4E70E94AD2F84E08093620081E0809345
:1025F0006300882780936400E2E2F4E70E94AD2F35
:1026000086E08093620081E0809363008827809356
:102610006400E4E3F4E70E94AD2F06B347E004232F
:10262000A5E6B0E00C9300916500053011F00C9424
:102630001B130C941F130E944B2F0C940D130E941C
:10264000EF2080E080935001009150010F3718F087
:1026500011F00C94521380E3809396000091960041
:102660000A3318F011F00C944613A0E5B1E04C9138
:10267000A6E9B0E05C9191E00E94DA31A6E9B0E011
:102680008C918F5F8C9310F40C942E138AE090E061
:102690000E941D30A0E5B1E08C918F5F8C9310F407
:1026A0000C9424130E947C3100914F01023011F0F0
:1026B0000C94831381E08093620081E08093630037
:1026C000882780936400E8E4F4E70E94AD2F83E05C
:1026D0008093620081E08093630088278093640088
:1026E000EAE5F4E70E94AD2F84E08093620081E088
:1026F00080936300882780936400ECE6F4E70E94EF
:10270000AD2F0C94DB13063011F00C94B01381E064
:102710008093620081E08093630088278093640047
:10272000E8E4F4E70E94AD2F83E08093620081E04B
:1027300080936300882780936400EAE5F4E70E94B1
:10274000AD2F84E08093620081E08093630088274E
:1027500080936400ECE6F4E70E94AD2F0C94DB1349
:10276000073011F00C94DB1381E08093620081E06C
:1027700080936300882780936400E8E4F4E70E9474
:10278000AD2F83E08093620081E08093630088270F
:1027900080936400EAE5F4E70E94AD2F84E0809323
:1027A000620081E080936300882780936400ECE6F8
:1027B000F4E70E94AD2FE2E0F0E00E94B42FA3E521
:1027C000B2E0E0E8F0E00E948236A6EDB3E00D93BF
:1027D0001C930E947C3181E08093620081E08093B1
:1027E0006300882780936400E8E4F4E70E94AD2F3B
:1027F00085E08093620081E0809363008827809366
:102800006400ECE6F1E70E94AD2FE0ECF3E0A0E617
:10281000B0E0ED93FC9386E08093620081E08093CA
:102820006300882780936400EEE7F4E70E94AD2FF1
:10283000A0EEB6E0E8EDF3E00E94E1350E94A52F9E
:1028400087E08093620081E0809363008827809313
:102850006400E6E8F4E70E94AD2FA0EEB6E0E6EDF6
:10286000F3E00E94E1350E94A52FA6EDB3E00D91A3
:102870001C91A8EDB3E04D915C91041B150BA4EEE7
:10288000B3E00D931C93E4EBF0E70E946234E4EEB6
:10289000F3E0D190E080FF2400270E941E330E94C5
:1028A000C633EDE0F0E0ACEDB3E00E943F36E0EC83
:1028B000F0E70E946234E4EEF3E0D190E080FF2480
:1028C00000270E941E330E947033EDE0F0E0A6EE78
:1028D000B3E00E943F36E0ECF0E70E946234ECED9A
:1028E000F3E00E94FA320E947033EDE0F0E0A0EED7
:1028F000B3E00E943F36E0ECF3E0A0E6B0E0ED93F9
:10290000FC9388E08093620081E0809363008827D5
:1029100080936400EEE8F4E70E94AD2FECEDF3E065
:102920000E943737DD2CEE2CFF2C002FA0EEB6E0F6
:10293000EDE0F0E00E94FA320E942C300E94A52FB8
:10294000E6E9F4E70E94AD2FE2E0F0E00E94B42F48
:1029500000914F01053011F00C94531580E890E080
:10296000A0E4B4E08D939C93ACECB0E00D911D918C
:102970002D913C91A8ECB0E04D915D916D917C91D1
:102980000E94C935AEEEB0E00D931D932D933D939B
:10299000A0E4B4E00D911C912227332749EF54E1C4
:1029A00060E070E00E946E32A7E3B4E00D931D93E7
:1029B0002D933D93AEEEB0E04D915D916D917C9184
:1029C000A7E3B4E00D911D912D913C910E94CE356D
:1029D0001CF011F00C940C1502E010E0A0E4B4E03F
:1029E0004D915C910E946432A0E4B4E00D931C937D
:1029F000A0E4B4E00D911C912227332749EF54E164
:102A000060E070E00E946E32A7E3B4E00D931D9386
:102A10002D933D930C94DA14AEEEB0E00D911D9120
:102A20002D913C91A0E4B4E04D915C91662777270D
:102A30000E94C02FA7E3B4E04D935D936D937D9307
:102A4000A0E4B4E00D911C9140E850E00E948B2F6F
:102A5000ABE3B4E04D935C93ABE3B4E00D911C9118
:102A6000013050E0150718F011F00C9439150C9452
:102A70004715ABE3B4E00D911C9142E050E00E9499
:102A80008B2FABE2B4E04D935C930C944F15ABE30A
:102A9000B4E08D919C91ABE2B4E08D939C93A1E363
:102AA000B4E00E945D350E947C3187E090E0AEEE9C
:102AB000B3E08D939C93AAEEB3E00E945D3580E075
:102AC000809350017091E8007B7F7093E800E0EC08
:102AD000F3E0A0E6B0E0ED93FC9306B347E00423F7
:102AE000A5E6B0E00C93A0E5B1E08C918F5F8C93EC
:102AF000009150010F3718F011F00C9481150C94CF
:102B0000331980E080935001A8EEB0E08C9182FBF5
:102B100016F00C9492157091E8007B7F7093E8009A
:102B20000E947C31AAEEB3E08C918A9380E08A9374
:102B3000AAEEB3E08C918A938FE38A9381E08A9323
:102B40000E94013280E08A93AEEEB3E08C918A93CA
:102B50008FE78A93AEEEB3E08C918A9381E08A93FB
:102B60000E9401320E94A52D00914F01053011F005
:102B70000C94E21581E08093620081E08093630011
:102B8000882780936400E8EFF2E70E94AD2F81E090
:102B90008093620081E080936300882780936400C3
:102BA000A4E3B1E00E94A72FEAE9F4E70E94AD2F69
:102BB000A5EFB3E00E94A72FEEE9F4E70E94AD2F46
:102BC0000C94081688E08093620081E08093630093
:102BD000882780936400E8EFF2E70E94AD2F88E039
:102BE0008093620081E08093630088278093640073
:102BF000A4E3B1E00E94A72FEAE9F4E70E94AD2F19
:102C0000A5EFB3E00E94A72FEEE9F4E70E94AD2FF5
:102C100000914F01073011F00C94C6167091E80036
:102C200070647093E800E1EFF3E00E94FA32E4ECA4
:102C3000F0E70E9462340E946B3410F40C94281662
:102C4000A4E3B1E0E2EAF4E70E9491320C94A81602
:102C5000A5EFB3E00E948134EDE0F0E0AEEFB3E029
:102C60000E943F36E8ECF0E70E946234EEEFF3E0BA
:102C70000E94FA320E94C633EDE0F0E0AEEFB3E01E
:102C80000E943F36ECECF0E70E946234EEEFF3E096
:102C90000E94FA320E947033EDE0F0E0AEEFB3E054
:102CA0000E943F36EEEFF3E00E94FF32ECE9F0E7DE
:102CB0000E9459340E94D737EDE0F0E0A2E0B4E082
:102CC0000E943F36E8E9F0E70E946234E2E0F4E077
:102CD0000E94FA320E940734EDE0F0E0AEEFB3E07C
:102CE0000E943F36E8E9F0E70E946234E2E0F4E057
:102CF0000E94FA320E94F833EDE0F0E0A2E0B4E086
:102D00000E943F36E2E0F4E00E94FF32EEEFF3E093
:102D10000E94FA320E947033EDE0F0E0AEEFB3E0D3
:102D20000E943F36A0EEB6E0AF93BF93EEEFF3E024
:102D30000E94FA320E942C3011E002E0BF91AF9164
:102D40000E947C35E0EEF6E0A4E3B1E00E943A3662
:102D500081E08093620081E0809363008827809304
:102D60006400E8EFF2E70E94AD2F81E080936200FB
:102D700081E080936300882780936400E6EAF4E7AB
:102D80000E94AD2FA4E3B1E00E94A72F00914F0154
:102D9000023011F00C942A19A3E5B1E0E0E8F0E06C
:102DA0000E949A36ABE2B4E00D931C93A3E3B4E027
:102DB0004D935C9387E08093620081E08093630091
:102DC000882780936400E2EBF4E70E94AD2FA0EE29
:102DD000B6E0EBE2F4E00E94E1350E94A52F86E028
:102DE0008093620081E08093630088278093640071
:102DF000E8EBF4E70E94AD2FA0EEB6E0E3E3F4E0E9
:102E00000E94E1350E94A52FABE2B4E00D911C9128
:102E10004FE050E0040F151FA1E3B4E00D931C93A5
:102E200080913304809396004091960001E004174E
:102E300018F011F00C943E17A1E3B4E04D915C91B1
:102E4000A6E9B0E0AD90BB24A1E5B1E0AA0CBB1CA3
:102E5000AA0DBB1D0D911C910417150718F011F058
:102E60000C9434170C9436170C943E1780919600EE
:102E700081508093960010F00C9414178091960066
:102E800080933504809133048093960000919600DE
:102E90000F3718F011F00C946F17A1E3B4E04D91C7
:102EA0005C91A6E9B0E0AD90BB24A1E5B1E0AA0C2D
:102EB000BB1CAA0DBB1D0D911C910417150718F022
:102EC00011F00C9465170C9467170C946F17A6E912
:102ED000B0E08C918F5F8C9310F40C944617809126
:102EE000960080933604A6E3B4E00C9111272227C4
:102EF0003327A5E3B4E04C915527662777270E9436
:102F0000C935A7E3B4E00D931D932D933D93A7E33B
:102F1000B4E00D911D912D913C91A0E7B0E04D9151
:102F20005D916D917C910E946E32A7E3B4E00D93A8
:102F30001D932D933D930091360440913504040F69
:102F4000A5E3B4E00C93A5E3B4E00C9142E00E9449
:102F500072360C93E3E3F4E0D190E080FF24002785
:102F60000E941E330E9455332F933F934F935F93DC
:102F7000E0E7F0E00E94FA320E941E335F914F9129
:102F80003F912F910E94C633EDE0F0E0A7E2B4E05C
:102F90000E943F36E7E2F4E00E94FF32E8ECF0E006
:102FA0000E94FA320E941E330E940734EDE0F0E0E6
:102FB000A7E2B4E00E943F36E2E9F0E00E94FA3274
:102FC0000E941E330E945533E7E2F4E00E94FA3279
:102FD0000E947033EDE0F0E0ABE4B1E00E943F36D8
:102FE000A0EEB6E0AF93BF93EBE4F1E00E94FA32BB
:102FF0000E942C3011E005E0BF91AF910E947C351A
:10300000E0EEF6E0A4E3B1E00E943A3687E0809378
:10301000620081E080936300882780936400EEEB78
:10302000F4E70E94AD2FA4E3B1E00E94A72FE2ECE9
:10303000F4E70E94AD2FE2E9F0E00E94FA320E942C
:103040001E330E9455332F933F934F935F93E7E3D3
:10305000F4E00E94FA320E941E335F914F913F913B
:103060002F910E947033EDE0F0E0A7E2B4E00E94FF
:103070003F36E7E2F4E00E94FF32EBE4F1E00E9429
:10308000FA320E947033EDE0F0E0A7E2B4E00E9473
:103090003F36E7E2F4E00E943737EDE0F0E0A7E2E8
:1030A000B4E00E943F3684E08093620081E0809328
:1030B0006300882780936400E6ECF4E70E94AD2F5C
:1030C000A0EEB6E0E7E2F4E00E94FA320E942C3073
:1030D0000E94A52FEBE4F1E00E94FF32EBE4F1E067
:1030E0000E94FA320E94C633EDE0F0E0ABE4B1E0BA
:1030F0000E943F36E0EDF0E70E946234EBE4F1E03D
:103100000E94FA320E94C633EDE0F0E0ABE4B1E099
:103110000E943F36EEE1F4E00E94FF32EBE4F1E082
:103120000E94FA320E94C633EDE0F0E0A7E2B4E07C
:103130000E943F36E4EDF0E70E946234E7E2F4E0FB
:103140000E94FA320E94C633EDE0F0E0A7E2B4E05C
:103150000E943F36E7E2F4E00E94FF32E8E9F0E740
:103160000E9459340E947033EDE0F0E0A7E2B4E031
:103170000E943F36A0EEB6E0AF93BF93E7E2F4E0E3
:103180000E94FA320E942C3011E001E0BF91AF9111
:103190000E947C35E0EEF6E0A4E3B1E00E943A360E
:1031A00085E08093620081E08093630088278093AC
:1031B0006400EAECF4E70E94AD2FA4E3B1E00E94C2
:1031C000A72FEEECF4E70E94AD2FEAE1F4E00E94B5
:1031D000FF32EBE4F1E00E94FA320E94C633EDE0E8
:1031E000F0E0A7E2B4E00E943F36E7E2F4E00E949C
:1031F000FF32E8EDF0E70E9459340E947033EDE0B1
:10320000F0E0A7E2B4E00E943F36E7E2F4E00E947B
:103210003737EDE0F0E0A7E2B4E00E943F3686E009
:103220008093620081E0809363008827809364002C
:10323000E2EDF4E70E94AD2FA0EEB6E0E7E2F4E0A5
:103240000E94FA320E942C300E94A52FE6EDF4E78E
:103250000E94AD2FA8EEB0E08C9185FB16F00C9487
:1032600033190E94A52D00914F01053011F40C94E3
:10327000D21941E050E060E070E0A8EDB0E00D91BF
:103280001D912D913C910E94CE3511F00C947C192A
:10329000EAEEF0E00E94FA320E941E330E9455339B
:1032A0002F933F934F935F93E0E5F1E0D080EE24BE
:1032B000FF2400270E941E335F914F913F912F9171
:1032C0000E94C633EDE0F0E0AEEFB0E00E943F3682
:1032D000EEEFF0E00E94FF32E8ECF0E00E94FA32FC
:1032E0000E941E330E940734EDE0F0E0AEEFB0E044
:1032F0000E943F360C94BC19E0E5F1E0D080EE244A
:10330000FF2400270E941E330E945533E2EFF0E0B5
:103310000E94FA320E94C633EDE0F0E0AAEFB0E07E
:103320000E943F36E6EFF0E00E94FF32EAEFF0E065
:103330000E94FA320E940734EDE0F0E0AAEFB0E01C
:103340000E943F36EAEFF0E00E94FF32ECE9F0E73E
:103350000E9459340E94D737EDE0F0E0AAEFB0E0C8
:103360000E943F36EAEFF0E00E943737EDE0F0E0F0
:10337000AEEFB0E00E943F360E94722200915001F1
:10338000003011F00C94CA1985E090E00E941D30C5
:103390000C94D219EF93FF93ECE8F1E00E94143003
:1033A000FF91EF910091500141E0040FA1E5B1E0E0
:1033B0000C9300914F01053011F00C941F1B0091EC
:1033C0005001013081E008F480E08F9300915001BA
:1033D0000E3781E010F009F080E09F918923882367
:1033E00011F40C94841AA1E5B1E0AD90BB24A1E5E1
:1033F000B1E0AA0CBB1CAA0DBB1D0E945D3581E08B
:1034000080939600ABE3B4E04D915C91A6E9B0E007
:103410000D9111270417150718F011F00C94821A5A
:10342000E7E3F4E00E94FA320E941E330E94553313
:103430002F933F934F935F93E1E3F4E0D190E080CB
:10344000FF2400270E941E335F914F913F912F91DF
:103450000E94C633EDE0F0E0AEEFB0E00E943F36F0
:10346000EEEFF0E00E94FF32E8ECF0E00E94FA326A
:103470000E941E330E940734EDE0F0E0AEEFB0E0B2
:103480000E943F360E947222A1E3B4E00E94572FAF
:1034900007B1007E066007B90E949732A0E4B4E04D
:1034A0008D939C93A1E5B1E0AD90BB24A1E5B1E083
:1034B000AA0CBB1CAA0DBB1D4D915C91A0E4B4E00D
:1034C0000D911C910417150718F011F00C946A1A4D
:1034D0000C947A1AA0E4B4E08D919C91A1E5B1E03E
:1034E000AD90BB24A1E5B1E0AA0CBB1CAA0DBB1D8D
:1034F0008D939C93A6E9B0E08C918F5F8C9310F430
:103500000C94021A0C941D1BA1E5B1E0AD90BB24F4
:10351000A1E5B1E0AA0CBB1CAA0DBB1D0E945D3544
:1035200081E080939600ABE2B4E04D915C91A6E916
:10353000B0E00D9111270417150718F011F00C9445
:10354000131BE7E3F4E00E94FA320E941E330E944C
:1035500055332F933F934F935F93E1E3F4E0D19082
:10356000E080FF2400270E941E335F914F913F911E
:103570002F910E94C633EDE0F0E0AEEFB0E00E9484
:103580003F36EEEFF0E00E94FF32E8ECF0E00E9400
:10359000FA320E941E330E940734EDE0F0E0AEEFF5
:1035A000B0E00E943F360E947222A1E3B4E00E9484
:1035B000572F07B1007E066007B90E949732A0E43A
:1035C000B4E08D939C93A1E5B1E0AD90BB24A1E55F
:1035D000B1E0AA0CBB1CAA0DBB1D4D915C91A0E4EF
:1035E000B4E00D911C910417150718F011F00C941C
:1035F000FB1A0C940B1BA0E4B4E08D919C91A1E507
:10360000B1E0AD90BB24A1E5B1E0AA0CBB1CAA0DB2
:10361000BB1D8D939C93A6E9B0E08C918F5F8C933A
:1036200010F40C94931A009150010F3711F00C9480
:103630001D1BA1E3B4E00E945D350C94311B07B162
:10364000007E066007B90E949732A1E5B1E0AD9017
:10365000BB24A1E5B1E0AA0CBB1CAA0DBB1D8D9338
:103660009C93A1E5B1E0AD90BB24A1E5B2E0AA0C2A
:10367000BB1CAA0DBB1D4D915C91A1E5B1E0AD90C5
:10368000BB24A1E5B1E0AA0CBB1CAA0DBB1D0D918A
:103690001C910417150718F011F00C94511B0C9491
:1036A000691BA1E5B1E0AD90BB24A1E5B2E0AA0C95
:1036B000BB1CAA0DBB1D8D919C91A1E5B1E0AD9005
:1036C000BB24A1E5B1E0AA0CBB1CAA0DBB1D8D93C8
:1036D0009C93A8EDB3E04D915C91A1E5B1E0AD9074
:1036E000BB24A1E5B1E0AA0CBB1CAA0DBB1D0D912A
:1036F0001C910417150710F00C948E1BA8EDB3E075
:103700008D919C91A1E5B1E0AD90BB24A1E5B1E024
:10371000AA0CBB1CAA0DBB1D8D939C93A1E5B1E027
:10372000AD90BB24A1E5B2E0AA0CBB1CAA0DBB1D49
:103730000D911C91A1E5B1E0AD90BB24A1E5B1E0F4
:10374000AA0CBB1CAA0DBB1D4D915C91041B150B53
:10375000AAEFB3E00D931C93E6EEF3E00E94FF3274
:10376000EAEFF3E0D190E080FF2400270E941E33AF
:103770000E947033EDE0F0E0ABE4B1E00E943F3630
:10378000EBE4F1E00E943737EDE0F0E00E94BC325C
:10379000AAEFB3E0DD92EC92AAEFB3E00D911C9199
:1037A00047E050E0040F151FAAEFB3E00D931C9300
:1037B000AAEFB3E00D911C91003050E0150710F016
:1037C0000C94E61BAAEFB3E00E945D35AAEFB3E0CC
:1037D0000D911C910F3350E0150718F011F00C9467
:1037E000F31B0C94F91B8FE390E0AAEFB3E08D93E9
:1037F0009C9300914F01053011F00C94321C0FE79F
:1038000040915001041BA2E5B1E00C93A2E5B1E0A8
:103810008C918A938FE38A93A2E5B1E08C918A938D
:10382000A1E5B1E0AD90BB24A2E5B3E0AA0DBB1DBC
:103830008C918A9380E08A930E940132A2E5B1E0E4
:103840008C918A938FE38A93A2E5B1E08C918A935D
:10385000AAEFB3E08C918A9381E08A930E940132AF
:103860000C944A1CA0E5B1E04C91A1E5B1E0AD900B
:10387000BB24A2E5B3E0AA0DBB1D5C9190E00E94C1
:10388000DA31A0E5B1E04C91AAEFB3E05C9191E0B0
:103890000E94DA318091FA03A1E5B1E0AD90BB243A
:1038A000A2E5B3E0AA0DBB1D8C9300916500053025
:1038B00011F00C94631C0E944B2F8AEF90E00E9441
:1038C0001D300C94820500916500033011F00C94BA
:1038D000DD1D0E944B2FAAEEB3E08C918A9380E00D
:1038E0008A93AAEEB3E08C918A938FE38A9380E067
:1038F0008A930E940132AAEEB3E00E945E2FAAEEE4
:10390000B3E00D911C91003050E015070CF402C09B
:103910000C94091DAAEEB3E00E945D357091E80099
:1039200074607093E800ACECB0E00D911D912D91A6
:103930003C91A8ECB0E04D915D916D917C910E941D
:10394000C935ACE6B0E00D931D932D933D93ACE6E5
:10395000B0E00D911D912D913C914AE050E060E066
:1039600070E00E94C02FACE6B0E04D935D936D9384
:103970007D93A8ECB0E00D911D912D913C91ACE6AA
:10398000B0E04D915D916D917C910E94C935A8EC9C
:10399000B0E00D931D932D933D93A0ECB0E04D91BD
:1039A0005D916D917C91A8ECB0E00D911D912D91F0
:1039B0003C910E94CE350CF402C00C94F51CA8EC8E
:1039C000B0E00D911D912D913C91ACE6B0E04D9190
:1039D0005D916D917C910E94C435A8ECB0E00D938F
:1039E0001D932D933D930C94091DACECB0E00D910B
:1039F0001D912D913C91ACE6B0E04D915D916D91A2
:103A00007C910E94C935ACECB0E00D931D932D93D1
:103A10003D93AAEEB3E08C918A9380E08A93AAEE5C
:103A2000B3E08C918A938FE38A9381E08A930E941A
:103A3000013280E08A93AEEEB3E08C918A938FE7F7
:103A40008A93AEEEB3E08C918A9381E08A930E94D0
:103A5000013200914F01053011F40C94501D80E0AB
:103A60008093F0030091F0030F3718F011F00C94DD
:103A7000501DA0EFB3E04C91A0EFB3E0AD90BB249C
:103A8000A3E5B3E0AA0DBB1D5C9191E00E94DA3181
:103A9000A0EFB3E08C918F5F8C9310F40C94321DE7
:103AA00000914F01053011F00C94881DEAEEF0E012
:103AB0000E94FA320E941E330E9455332F933F9387
:103AC0004F935F93E2E5F1E0D080EE24FF240027DE
:103AD0000E941E335F914F913F912F910E94C633F8
:103AE000EDE0F0E0AEEFB0E00E943F36EEEFF0E048
:103AF0000E94FF32E8ECF0E00E94FA320E941E338E
:103B00000E940734EDE0F0E0AEEFB0E00E943F36F7
:103B10000E94A52D00914F01053011F00C94AB1DB2
:103B200081E08093620081E0809363008827809326
:103B30006400A4E3B1E00E94A72FEAEDF4E70E943D
:103B4000AD2FA5EFB3E00E94A72FEEE9F4E70E94A6
:103B5000AD2F0C94C41D88E08093620081E08093B7
:103B60006300882780936400A4E3B1E00E94A72F3C
:103B7000EAEDF4E70E94AD2FA5EFB3E00E94A72F76
:103B8000EEE9F4E70E94AD2F84E690E00E941D303C
:103B900006B347E00423A5E6B0E00C93009165006E
:103BA000033011F00C94D81D0E944B2F0C946B1C09
:103BB0007091E80070627093E80000916500013038
:103BC00011F00C945B1F0E944B2FAAEEB3E08C9176
:103BD0008A9380E08A93AAEEB3E08C918A938FE374
:103BE0008A9380E08A930E940132AAEEB3E00E9499
:103BF000572FAAEEB3E00D911C910F3750E0150737
:103C00001CF011F00C94061E0C94891E8FE790E0B6
:103C1000AAEEB3E08D939C937091E800746070936A
:103C2000E800ACECB0E00D911D912D913C91A8EC19
:103C3000B0E04D915D916D917C910E94C935ACE6EB
:103C4000B0E00D931D932D933D93ACE6B0E00D9144
:103C50001D912D913C914AE050E060E070E00E949F
:103C6000C02FACE6B0E04D935D936D937D93ACECCB
:103C7000B0E00D911D912D913C91ACE6B0E04D91DD
:103C80005D916D917C910E94C435ACECB0E00D93D8
:103C90001D932D933D93ACEBB0E04D915D916D91F3
:103CA0007C91ACECB0E00D911D912D913C910E9466
:103CB000CE351CF011F00C945F1E0C94751EACEC0C
:103CC000B0E00D911D912D913C91ACE6B0E04D918D
:103CD0005D916D917C910E94C935ACECB0E00D9383
:103CE0001D932D933D930C94891EA8ECB0E00D918B
:103CF0001D912D913C91ACE6B0E04D915D916D919F
:103D00007C910E94C435A8ECB0E00D931D932D93D7
:103D10003D93AAEEB3E08C918A9380E08A93AAEE59
:103D2000B3E08C918A938FE38A9381E08A930E9417
:103D3000013280E08A93AEEEB3E08C918A938FE7F4
:103D40008A93AEEEB3E08C918A9381E08A930E94CD
:103D5000013200914F01053011F40C94D01E80E027
:103D60008093F0030091F0030F3718F011F00C94DA
:103D7000D01EA0EFB3E04C91A0EFB3E0AD90BB2418
:103D8000A3E5B3E0AA0DBB1D5C9191E00E94DA317E
:103D9000A0EFB3E08C918F5F8C9310F40C94B21E63
:103DA00000914F01053011F00C94081FEAEEF0E08D
:103DB0000E94FA320E941E330E9455332F933F9384
:103DC0004F935F93E2E5F1E0D080EE24FF240027DB
:103DD0000E941E335F914F913F912F910E94C633F5
:103DE000EDE0F0E0AEEFB0E00E943F36EEEFF0E045
:103DF0000E94FF32E8ECF0E00E94FA320E941E338B
:103E00000E940734EDE0F0E0AEEFB0E00E943F36F4
:103E10000E94A52D00914F01053011F00C942B1F2D
:103E200081E08093620081E0809363008827809323
:103E30006400A4E3B1E00E94A72FEAEDF4E70E943A
:103E4000AD2FA5EFB3E00E94A72FEEE9F4E70E94A3
:103E5000AD2F0C94441F88E08093620081E0809332
:103E60006300882780936400A4E3B1E00E94A72F39
:103E7000EAEDF4E70E94AD2FA5EFB3E00E94A72F73
:103E8000EEE9F4E70E94AD2F84E690E00E941D3039
:103E900006B347E00423A5E6B0E00C93009165006B
:103EA000013011F00C94561F0C94E51D7091E80040
:103EB00070627093E80000916500043011F00C947A
:103EC00024200E944B2F80E08A93AEEEB3E08C91C9
:103ED0008A938FE78A93AEEEB3E08C918A9380E069
:103EE0008A930E940132AEEEB3E00E94572FAEEEED
:103EF000B3E00D911C910F3350E015071CF011F049
:103F00000C94841F0C948A1F8FE390E0AEEEB3E014
:103F10008D939C9380E08A93AEEEB3E08C918A936C
:103F20008FE78A93AEEEB3E08C918A9381E08A9317
:103F30000E940132AAEEB3E08C918A9380E08A93CA
:103F4000AAEEB3E08C918A938FE38A9381E08A93FF
:103F50000E94013200914F01053011F40C94D11FE1
:103F600080E08093F0030091F0030F3718F011F018
:103F70000C94D11FA0EFB3E04C91A0EFB3E0AD9053
:103F8000BB24A3E5B3E0AA0DBB1D5C9191E00E94A8
:103F9000DA31A0EFB3E08C918F5F8C9310F40C9426
:103FA000B31F0E94A52D00914F01053011F00C9414
:103FB000F41F81E08093620081E080936300882792
:103FC00080936400A4E3B1E00E94A72FEAEDF4E738
:103FD0000E94AD2FA5EFB3E00E94A72FEEE9F4E712
:103FE0000E94AD2F0C940D2088E08093620081E048
:103FF00080936300882780936400A4E3B1E00E946B
:10400000A72FEAEDF4E70E94AD2FA5EFB3E00E94E1
:10401000A72FEEE9F4E70E94AD2F84E690E00E941E
:104020001D3006B347E00423A5E6B0E00C930091F1
:104030006500043011F00C941F200C94631F7091E4
:10404000E80070627093E80000916500063011F09E
:104050000C94EB200E944B2F80E08A93AEEEB3E0ED
:104060008C918A938FE78A93AEEEB3E08C918A931A
:1040700080E08A930E940132AEEEB3E00E945E2F90
:10408000AEEEB3E00D911C91003050E015070CF43A
:1040900002C00C944F20AEEEB3E00E945D3580E08C
:1040A0008A93AEEEB3E08C918A938FE78A93AEEE5B
:1040B000B3E08C918A9381E08A930E940132AAEE48
:1040C000B3E08C918A9380E08A93AAEEB3E08C915E
:1040D0008A938FE38A9381E08A930E940132009150
:1040E0004F01053011F40C94962080E08093F0038A
:1040F0000091F0030F3718F011F00C949620A0EF08
:10410000B3E04C91A0EFB3E0AD90BB24A3E5B3E0E6
:10411000AA0DBB1D5C9191E00E94DA31A0EFB3E0E3
:104120008C918F5F8C9310F40C9478200E94A52DB5
:1041300000914F01053011F00C94B92081E080937B
:10414000620081E080936300882780936400A4E389
:10415000B1E00E94A72FEAEDF4E70E94AD2FA5EF92
:10416000B3E00E94A72FEEE9F4E70E94AD2F0C9474
:10417000D22088E08093620081E0809363008827EA
:1041800080936400A4E3B1E00E94A72FEAEDF4E776
:104190000E94AD2FA5EFB3E00E94A72FEEE9F4E750
:1041A0000E94AD2F84E690E00E941D3006B347E0E8
:1041B0000423A5E6B0E00C9300916500063011F0F1
:1041C0000C94E6200E944B2F0C942C207091E80058
:1041D00070627093E8000C946D150C948F050E942A
:1041E000DD2181E08093420400914204003818F000
:1041F00011F00C949E2141E050E060E070E0A8EDE9
:10420000B0E00D911D912D913C910E94CE3511F0A1
:104210000C943E21EAEEF0E00E94FA320E941E3336
:104220000E9455332F933F934F935F93E2E4F4E062
:10423000D080EE24FF2400270E941E335F914F910F
:104240003F912F910E94C633EDE0F0E0AEEFB0E079
:104250000E943F36EEEFF0E00E94FF32E8ECF0E023
:104260000E94FA320E941E330E940734EDE0F0E013
:10427000AEEFB0E00E943F360C947E21E2E4F4E021
:10428000D080EE24FF2400270E941E330E94553365
:10429000E2EFF0E00E94FA320E94C633EDE0F0E077
:1042A000AAEFB0E00E943F36E6EFF0E00E94FF3256
:1042B000EAEFF0E00E94FA320E940734EDE0F0E00D
:1042C000AAEFB0E00E943F36EAEFF0E00E94FF3232
:1042D000ECE9F0E70E9459340E94D737EDE0F0E0B6
:1042E000AAEFB0E00E943F36EAEFF0E00E943737D5
:1042F000EDE0F0E0AEEFB0E00E943F360E947222A7
:1043000081E090E00E941D3007B1007E066007B991
:104310000E949732A2E4B4E0AD90BB24A1E5B2E0E4
:10432000AA0CBB1CAA0DBB1D8D939C93A2E4B4E008
:104330008C918F5F8C9310F40C94F4200895A881D5
:10434000B9818D919C91A5E4B4E08D939C93939851
:1043500081E08093470400914704003118F011F088
:104360000C94DB21A5E4B4E00D911C9140E050E8F1
:1043700004231523A3E4B4E00D931C93A3E4B4E059
:104380000D911C91003050E8150711F00C94CB21D1
:10439000959A0C94CC2195989498949A91E0A5E4E0
:1043A000B4E00E94A032A7E4B4E08C918F5F8C93BC
:1043B00010F40C94AB21939A0895ACECB0E04D91BD
:1043C0005D916D917C91A8ECB0E00D911D912D91C6
:1043D0003C910E94CE3511F00C94F421AEEEB0E089
:1043E0000E945F350C947122ACECB0E00D911D91F0
:1043F0002D913C91A8ECB0E04D915D916D917C9137
:104400000E94C935AAEEB0E00D931D932D933D9304
:10441000AAEEB0E00D911D912D913C9140E850E045
:1044200060E070E00E94C02FAAEEB0E04D935D9373
:104430006D937D9342E050E060E070E0A8EDB0E065
:104440000D911D912D913C910E94CE3511F00C944F
:104450007122ECECF0E00E94FA320E941E33A2EFCF
:10446000B0E00E945033E2EFF0E00E943D38EDE012
:10447000F0E0A2EFB0E00E943F36E8ECF0E00E94EE
:10448000FA320E941E33A6EFB0E00E945033E6EFEE
:10449000F0E00E943D38EDE0F0E0A6EFB0E00E94D1
:1044A0003F36E6EFF0E00E94FF32E2EFF0E00E94DC
:1044B000FA320E94F833EDE0F0E0A2EFB0E00E94A3
:1044C0003F36ECEDF0E70E946234E2EFF0E00E944C
:1044D000FA320E947033EDE0F0E0A2EFB0E00E940B
:1044E0003F360895EEEFF0E00E94BC32ACE4B4E059
:1044F000EDE0FF270E943F36ACE4B4E00D911C9143
:104500004FEF5FE304231523AAE4B4E00D931C935B
:1045100081E080935004009150040E3018F011F0A7
:104520000C949F2291E0ACE4B4E00E94AB32A0E591
:10453000B4E08C918F5F8C9310F40C948B22ACE4DC
:10454000B4E00D911C914FEF5FE304231523A8E421
:10455000B4E00D931C93A8E4B4E00D911C9140E0ED
:1045600050E4040F151FA8E4B4E00D931C93AAE4D3
:10457000B4E00D911C9140E050E4040F151FAAE433
:10458000B4E00D931C935A924A92A4E7B0E08D9147
:104590009C91D2018D939C9382E00E9460320E9494
:1045A0009F21229682E00E94532F5A924A92AAE4B7
:1045B000B4E08D919C91D2018D939C9382E00E94F6
:1045C00060320E949F21229682E00E94532F5A92CD
:1045D0004A92A8E4B4E08D919C91D2018D939C9372
:1045E00082E00E9460320E949F21229682E00E9417
:1045F000532F08950E947C3180E0809352048BE019
:104600008093510481E08093530400912A01023188
:1046100010F00C94382340912A01009151040417A2
:1046200011F00C94162381E080935204E4ECF0E046
:10463000A0E6B0E0ED93FC93A3E5B4E08C91809309
:10464000620081E080936300A2E5B4E08C918093E6
:104650006400ECEDF4E70E94AD2FE0ECF3E0A0E69F
:10466000B0E0ED93FC93A3E5B4E08C918F5F8C9365
:1046700080E080935204A1E5B4E08C918F5F8C932D
:1046800000912A01033110F00C94752340912A0106
:1046900000915104041711F00C94512381E0809390
:1046A0005204A3E5B4E08C918093620081E0809392
:1046B0006300A2E5B4E08C9180936400E6EEF4E739
:1046C0000E94AD2FABE2B1E00D91112746E050E022
:1046D0000E946432A0E0B1E0A00FB11F0E94A72F9A
:1046E000A3E5B4E08C918F5F8C9380E080935204BB
:1046F000A1E5B4E08C918F5F8C9300912A01043185
:1047000010F00C94082440912A01009151040417E0
:1047100011F00C948E2381E080935204E2E9F0E0E2
:104720000E94FA320E941E330E9455332F933F930A
:104730004F935F93E8ECF0E00E94FA320E941E3340
:104740005F914F913F912F910E947033EDE0F0E027
:10475000ABE4B1E00E943F36A0EEB6E0AF93BF936A
:10476000EBE4F1E00E94FA320E942C3011E004E008
:10477000BF91AF910E947C35E0EEF6E0A4E3B1E09A
:104780000E943A36EBE4F1E00E94FA32ECE9F0E7FD
:104790000E9462340E946B3410F00C94EA23A3E56B
:1047A000B4E08C918093620081E080936300A2E585
:1047B000B4E08C9180936400E2EFF4E70E94AD2FA7
:1047C000A4E3B1E00E94A72FE2ECF4E70E94AD2F32
:1047D0000C940324A3E5B4E08C918093620081E003
:1047E00080936300A2E5B4E08C9180936400EAEFCB
:1047F000F4E70E94AD2FA4E3B1E00E94A72FE2EC02
:10480000F4E70E94AD2FA3E5B4E08C918F5F8C9309
:1048100080E080935204A1E5B4E08C918F5F8C938B
:1048200040912A0100915104041711F00C941B24AB
:1048300081E080935204E2E9F0E00E94FA320E94A3
:104840001E330E9455332F933F934F935F93ECECAD
:10485000F0E00E94FA320E941E335F914F913F9127
:104860002F910E947033EDE0F0E0ABE4B1E00E94E4
:104870003F36A0EEB6E0AF93BF93EBE4F1E00E94C9
:10488000FA320E942C3011E004E0BF91AF910E94F7
:104890007C35E0EEF6E0A4E3B1E00E943A36EBE4CA
:1048A000F1E00E94FA32ECE9F0E70E9462340E94E3
:1048B0006B3410F00C947724A3E5B4E08C918093D2
:1048C000620081E080936300A2E5B4E08C91809364
:1048D0006400E2E0F5E70E94AD2FA4E3B1E00E949E
:1048E000A72FE2ECF4E70E94AD2F0C949024A3E5EF
:1048F000B4E08C918093620081E080936300A2E534
:10490000B4E08C9180936400EAE0F5E70E94AD2F5B
:10491000A4E3B1E00E94A72FE2ECF4E70E94AD2FE0
:1049200080E080935204A1E5B4E08C918F5F8C937A
:10493000A3E5B4E08C918F5F8C9340912A010091A4
:104940005104041711F00C94A82481E080935204C0
:1049500041E050E060E070E0A8EDB0E00D911D9105
:104960002D913C910E94CE3511F00C94BF24A2E40D
:10497000B1E0E2E1F5E70E9491320C94C524A2E493
:10498000B1E0E6E1F5E70E949132A3E5B4E08C9155
:104990008093620081E080936300A2E5B4E08C9193
:1049A00080936400EAE1F5E70E94AD2FA2E4B1E054
:1049B0000E94A72F80E0809352040E94DD21A1E590
:1049C000B4E08C918F5F8C93A3E5B4E08C918F5F02
:1049D0008C9340912A0100915104041711F00C941A
:1049E000F42481E08093520441E050E060E070E004
:1049F000A4EDB0E00D911D912D913C910E94CE351A
:104A000011F00C940B25A2E4B1E0E8E2F5E70E9476
:104A100091320C941125A2E4B1E0ECE2F5E70E949A
:104A20009132A3E5B4E08C918093620081E08093A1
:104A30006300A2E5B4E08C9180936400E0E3F5E7C5
:104A40000E94AD2FA2E4B1E00E94A72F80E08093E6
:104A50005204A1E5B4E08C918F5F8C93A3E5B4E0A0
:104A60008C918F5F8C9340912A010091510404171F
:104A700011F00C943E2581E080935204E2E9F0E0CD
:104A80000E94FA320E941E330E9455332F933F93A7
:104A90004F935F93E4ECF0E00E94FA320E941E33E1
:104AA0005F914F913F912F910E947033EDE0F0E0C4
:104AB000ABE4B1E00E943F36A0EEB6E0AF93BF9307
:104AC000EBE4F1E00E94FA320E942C3011E004E0A5
:104AD000BF91AF910E947C35E0EEF6E0A4E3B1E037
:104AE0000E943A36EBE4F1E00E94FA32ECE9F0E79A
:104AF0000E9462340E946B3410F00C949A25A3E556
:104B0000B4E08C918093620081E080936300A2E521
:104B1000B4E08C9180936400EEE3F5E70E94AD2F42
:104B2000A4E3B1E00E94A72FE2ECF4E70E94AD2FCE
:104B30000C94B325A3E5B4E08C918093620081E0EE
:104B400080936300A2E5B4E08C9180936400E6E476
:104B5000F5E70E94AD2FA4E3B1E00E94A72FE2EC9D
:104B6000F4E70E94AD2F80E080935204A1E5B4E009
:104B70008C918F5F8C93A3E5B4E08C918F5F8C93C5
:104B800040912A0100915104041711F00C94CB2597
:104B900081E08093520400912604013011F00C94BE
:104BA000E425A3E5B4E08C918093620081E08093DA
:104BB0006300A2E5B4E08C9180936400EEE4F5E735
:104BC0000E94AD2F0C943E26023011F00C94FB2570
:104BD000A3E5B4E08C918093620081E08093630050
:104BE000A2E5B4E08C9180936400E0E6F5E70E94D2
:104BF000AD2F0C943E26033011F00C941226A3E541
:104C0000B4E08C918093620081E080936300A2E520
:104C1000B4E08C9180936400E2E7F5E70E94AD2F49
:104C20000C943E26043011F00C942926A3E5B4E040
:104C30008C918093620081E080936300A2E5B4E0F0
:104C40008C9180936400E4E8F5E70E94AD2F0C940A
:104C50003E26053011F00C943E26A3E5B4E08C917D
:104C60008093620081E080936300A2E5B4E08C91C0
:104C700080936400E6E9F5E70E94AD2F80E0809321
:104C80005204A1E5B4E08C918F5F8C93A3E5B4E06E
:104C90008C918F5F8C9300912A01013118F011F0F3
:104CA0000C9454260C94972740912A0100915104AA
:104CB000041711F00C945F2681E080935204A0EE5B
:104CC000B6E0AF93BF93EAE1F4E00E94FA320E94AB
:104CD0002C3011E001E0BF91AF910E947C35E0EEF5
:104CE000F6E0A4E3B1E00E943A36EAE1F4E00E9483
:104CF000FA32ECE9F0E70E9462340E946B3410F063
:104D00000C949D26A3E5B4E08C918093620081E031
:104D100080936300A2E5B4E08C9180936400E8EA9C
:104D2000F5E70E94AD2FA4E3B1E00E94A72FEEECBF
:104D3000F4E70E94AD2F0C948F27EAE1F4E00E9483
:104D4000FA32ECE9F0E70E9462340E946B3481E0B1
:104D500008F480E08F93EAE1F4E00E94FA32E0EE9A
:104D6000F0E70E9462340E946B3481E010F009F099
:104D700080E09F918923882311F40C94DA26A3E51F
:104D8000B4E08C918093620081E080936300A2E59F
:104D9000B4E08C9180936400E4EBF5E70E94AD2FC2
:104DA000A4E3B1E00E94A72FEEECF4E70E94AD2F40
:104DB0000C948F27EAE1F4E00E94FA32E0EAF0E78F
:104DC0000E9462340E946B3481E008F480E08F938B
:104DD000EAE1F4E00E94FA32E4EEF0E70E94623485
:104DE0000E946B3481E010F009F080E09F918923EC
:104DF000882311F40C941727A3E5B4E08C918093D9
:104E0000620081E080936300A2E5B4E08C9180931E
:104E10006400E0ECF5E70E94AD2FA4E3B1E00E944E
:104E2000A72FEEECF4E70E94AD2F0C948F27EAE158
:104E3000F4E00E94FA32E4EAF0E70E9462340E9451
:104E40006B3481E008F480E08F93EAE1F4E00E94A3
:104E5000FA32E8EEF0E70E9462340E946B3481E09F
:104E600010F009F080E09F918923882311F40C94BD
:104E70005427A3E5B4E08C918093620081E0809395
:104E80006300A2E5B4E08C9180936400EAECF5E75E
:104E90000E94AD2FA4E3B1E00E94A72FEEECF4E74F
:104EA0000E94AD2F0C948F27EAE1F4E00E94FA32C1
:104EB000ECEEF0E70E9462340E946B3481E008F46B
:104EC00080E08F93EAE1F4E00E94FA32E0EFF0E74D
:104ED0000E9462340E946B3481E010F009F080E09F
:104EE0009F918923882311F40C948F27A3E5B4E0C4
:104EF0008C918093620081E080936300A2E5B4E02E
:104F00008C9180936400E4EDF5E70E94AD2FA4E35B
:104F1000B1E00E94A72FEEECF4E70E94AD2F80E0F5
:104F200080935204A3E5B4E08C918F5F8C93A1E54C
:104F3000B4E08C918F5F8C9300912A01023118F0BC
:104F400011F00C94A5270C94E82840912A010091B7
:104F50005104041711F00C94B02781E0809352049F
:104F6000A0EEB6E0AF93BF93EEE1F4E00E94FA3218
:104F70000E942C3011E001E0BF91AF910E947C357E
:104F8000E0EEF6E0A4E3B1E00E943A36EEE1F4E0B0
:104F90000E94FA32ECE9F0E70E9462340E946B341E
:104FA00010F00C94EE27A3E5B4E08C91809362009E
:104FB00081E080936300A2E5B4E08C91809364006B
:104FC000ECEDF5E70E94AD2FA4E3B1E00E94A72F1E
:104FD000E6EDF4E70E94AD2F0C94E028EEE1F4E05A
:104FE0000E94FA32ECE9F0E70E9462340E946B34CE
:104FF00081E008F480E08F93EEE1F4E00E94FA3261
:10500000E0EEF0E70E9462340E946B3481E010F021
:1050100009F080E09F918923882311F40C942B28B8
:10502000A3E5B4E08C918093620081E080936300FB
:10503000A2E5B4E08C9180936400E8EEF5E70E946D
:10504000AD2FA4E3B1E00E94A72FE6EDF4E70E94A4
:10505000AD2F0C94E028EEE1F4E00E94FA32E0EA91
:10506000F0E70E9462340E946B3481E008F480E033
:105070008F93EEE1F4E00E94FA32E4EEF0E70E9452
:1050800062340E946B3481E010F009F080E09F915F
:105090008923882311F40C946828A3E5B4E08C914B
:1050A0008093620081E080936300A2E5B4E08C917C
:1050B00080936400E4EFF5E70E94AD2FA4E3B1E034
:1050C0000E94A72FE6EDF4E70E94AD2F0C94E02894
:1050D000EEE1F4E00E94FA32E4EAF0E70E94623482
:1050E0000E946B3481E008F480E08F93EEE1F4E0FD
:1050F0000E94FA32E8EEF0E70E9462340E946B34BC
:1051000081E010F009F080E09F918923882311F459
:105110000C94A528A3E5B4E08C918093620081E013
:1051200080936300A2E5B4E08C9180936400EEEF7D
:10513000F5E70E94AD2FA4E3B1E00E94A72FE6EDB2
:10514000F4E70E94AD2F0C94E028EEE1F4E00E9419
:10515000FA32ECEEF0E70E9462340E946B3481E098
:1051600008F480E08F93EEE1F4E00E94FA32E0EF81
:10517000F0E70E9462340E946B3481E010F009F085
:1051800080E09F918923882311F40C94E028A3E503
:10519000B4E08C918093620081E080936300A2E58B
:1051A000B4E08C9180936400E8E0F6E70E94AD2FB4
:1051B000A4E3B1E00E94A72FE6EDF4E70E94AD2F33
:1051C00080E080935204A3E5B4E08C918F5F8C93D0
:1051D000A1E5B4E08C918F5F8C9300912A0103319B
:1051E00018F011F00C94F6280C94122940912A0121
:1051F00000915104041711F00C94012981E080936F
:105200005204A3E5B4E08C918093620081E0809326
:105210006300A2E5B4E08C9180936400E0E1F6E7DE
:105220000E94AD2F0E94DD21089500912A010C30CB
:1052300011F00C942E29ABE2B1E08C918F5F8C932E
:1052400000912B01063018F011F00C9429290C94D0
:105250002C2986E080932B010C943F2B0D3011F00C
:105260000C949729A8ECB0E00D911D912D913C91E3
:10527000ABE2B1E0AD90BB24AAE7B0E0AA0CBB1C46
:10528000AA0CBB1CAA0DBB1D4D915D916D917C912B
:105290000E94C435A8ECB0E00D931D932D933D936F
:1052A00042E050E060E070E0A4EDB0E00D911D91AF
:1052B0002D913C910E94CE3511F00C947529A8ECEB
:1052C000B0E00D911D912D913C91A4ECB0E04D9179
:1052D0005D916D917C910E94C435ACECB0E00D9372
:1052E0001D932D933D930C949529ACECB0E04D911A
:1052F0005D916D917C91A8ECB0E00D911D912D9187
:105300003C910E94CE351CF011F00C9489290C942C
:105310009529ACECB0E00D911D912D913C91A8EC3C
:10532000B0E00D931D932D933C930C943F2B0E30C6
:1053300011F00C94DB29ACECB0E00D911D912D9196
:105340003C91ABE2B1E0AD90BB24AAE7B0E0AA0C7F
:10535000BB1CAA0CBB1CAA0DBB1D4D915D916D9190
:105360007C910E94C435ACECB0E00D931D932D935D
:105370003D93ACEBB0E04D915D916D917C91ACECC7
:10538000B0E00D911D912D913C910E94CE351CF005
:1053900011F00C94CD290C94D929ACEBB0E00D910F
:1053A0001D912D913C91ACECB0E00D931D932D938C
:1053B0003C930C943F2B0F3011F00C94FE2941E0EC
:1053C00050E060E070E0A8EDB0E00D911D912D91EE
:1053D0003C910E94CE3511F00C94F629A8EDB0E076
:1053E000E4EFF0E70E9455350C94FC29A8EDB0E0FD
:1053F000ECEAF0E70E9455350C943F2B003111F098
:105400000C94572A41E050E060E070E0A4EDB0E079
:105410000D911D912D913C910E94CE3511F00C946F
:105420004F2AA4EDB0E0E4EFF0E70E945535A8EC78
:10543000B0E00D911D912D913C91A4ECB0E04D9107
:105440005D916D917C910E94C435ACECB0E00D9300
:105450001D932D933D93ACEBB0E04D915D916D911B
:105460007C91ACECB0E00D911D912D913C910E948E
:10547000CE351CF011F00C943F2A0C944B2AACEB67
:10548000B0E00D911D912D913C91ACECB0E00D93ED
:105490001D932D933C930E947C310C94552AA4EDCE
:1054A000B0E0ECEAF0E70E9455350C943F2B013157
:1054B00011F00C94BE2AA4ECB0E00D911D912D9139
:1054C0003C91ABE2B1E0AD90BB24AAE7B0E0AA0CFE
:1054D000BB1CAA0CBB1CAA0DBB1D4D915D916D910F
:1054E0007C910E94C435A4ECB0E00D931D932D93E4
:1054F0003D9342E050E060E070E0A4EDB0E00D913B
:105500001D912D913C910E94CE3511F00C94BC2A36
:10551000A8ECB0E00D911D912D913C91A4ECB0E070
:105520004D915D916D917C910E94C435ACECB0E0E1
:105530000D931D932D933D93ACEBB0E04D915D9198
:105540006D917C91ACECB0E00D911D912D913C9151
:105550000E94CE351CF011F00C94B02A0C94BC2A99
:10556000ACEBB0E00D911D912D913C91ACECB0E015
:105570000D931D932D933C930C943F2B023111F00E
:105580000C94D52AA6E2B4E08C918F5F8C930091A5
:105590002604053018F011F00C94D02A0C94D32A6C
:1055A00085E0809326040C943F2B033111F00C947A
:1055B0000B2BE6E2F4E0A190BB24E2E0F4E0AA0CBD
:1055C000BB1CAA0CBB1CEA0DFB1D0E94FF32EAE1CA
:1055D000F4E00E94FA320E940734EDE0F0E0AAE124
:1055E000B4E00E943F36EAE1F4E00E94FA32E8EFCC
:1055F000F0E70E9462340E946B3418F011F00C94B2
:10560000032B0C94092BAAE1B4E0E8EFF0E70E9429
:1056100055350C943F2B043111F00C943F2BE6E2EE
:10562000F4E0A190BB24E2E0F4E0AA0CBB1CAA0CBD
:10563000BB1CEA0DFB1D0E94FF32EEE1F4E00E946C
:10564000FA320E940734EDE0F0E0AEE1B4E00E94EF
:105650003F36EEE1F4E00E94FA32E8EFF0E70E9414
:1056600062340E946B3418F011F00C94392B0C94B6
:105670003F2BAEE1B4E0E8EFF0E70E945535089526
:1056800000912A010C3011F00C94562B80912B01C3
:10569000815080932B0100912B01013010F00C946C
:1056A000542B81E080932B010C94A42D0D3011F02C
:1056B0000C94BB2BA8ECB0E00D911D912D913C9169
:1056C000ABE2B1E0AD90BB24AAE7B0E0AA0CBB1CF2
:1056D000AA0CBB1CAA0DBB1D4D915D916D917C91D7
:1056E0000E94C935A8ECB0E00D931D932D933D9316
:1056F000A0ECB0E04D915D916D917C91A8ECB0E093
:105700000D911D912D913C910E94CE350CF402C05B
:105710000C94962BA0ECB0E00D911D912D913C9135
:10572000A8ECB0E00D931D932D933C9342E050E024
:1057300060E070E0A4EDB0E00D911D912D913C91E1
:105740000E94CE3511F00C94B92BA8ECB0E00D916D
:105750001D912D913C91A4ECB0E04D915D916D9126
:105760007C910E94C435ACECB0E00D931D932D9359
:105770003D930C94A42D0E3011F00C94FD2BACEC49
:10578000B0E00D911D912D913C91ABE2B1E0AD9057
:10579000BB24AAE7B0E0AA0CBB1CAA0CBB1CAA0D38
:1057A000BB1D4D915D916D917C910E94C935ACEC12
:1057B000B0E00D931D932D933D93A8ECB0E04D9177
:1057C0005D916D917C91ACECB0E00D911D912D91AE
:1057D0003C910E94CE350CF402C00C94FB2BA8EC3B
:1057E000B0E00D911D912D913C91ACECB0E00D938A
:1057F0001D932D933C930C94A42D0F3011F00C9419
:10580000202C41E050E060E070E0A8EDB0E00D91A8
:105810001D912D913C910E94CE3511F00C94182CC5
:10582000A8EDB0E0E4EFF0E70E9455350C941E2C93
:10583000A8EDB0E0ECEAF0E70E9455350C94A42DF9
:10584000003111F00C94792C41E050E060E070E000
:10585000A4EDB0E00D911D912D913C910E94CE35AB
:1058600011F00C94712CA4EDB0E0E4EFF0E70E948D
:105870005535A8ECB0E00D911D912D913C91A4EC13
:10588000B0E04D915D916D917C910E94C435ACEC7E
:10589000B0E00D931D932D933D93ACEBB0E04D9193
:1058A0005D916D917C91ACECB0E00D911D912D91CD
:1058B0003C910E94CE351CF011F00C94612C0C949C
:1058C0006D2CACEBB0E00D911D912D913C91ACECA9
:1058D000B0E00D931D932D933C930E947C310C946A
:1058E000772CA4EDB0E0ECEAF0E70E9455350C947B
:1058F000A42D013111F00C94122DABE2B1E0AD906A
:10590000BB24AAE7B0E0AA0CBB1CAA0CBB1CAA0DC6
:10591000BB1D4D915D916D917C91A4ECB0E00D911A
:105920001D912D913C910E94CE350CF402C00C9437
:10593000AF2CABE2B1E0AD90BB24AAE7B0E0AA0C7B
:10594000BB1CAA0CBB1CAA0DBB1D0D911D912D915A
:105950003C91A4ECB0E00D931D932D933C93A4ECEB
:10596000B0E00D911D912D913C91ABE2B1E0AD9075
:10597000BB24AAE7B0E0AA0CBB1CAA0CBB1CAA0D56
:10598000BB1D4D915D916D917C910E94C935A4EC38
:10599000B0E00D931D932D933D9342E050E060E005
:1059A00070E0A4EDB0E00D911D912D913C910E940D
:1059B000CE3511F00C94102DA8ECB0E00D911D9196
:1059C0002D913C91A4ECB0E04D915D916D917C9155
:1059D0000E94C435ACECB0E00D931D932D933D9324
:1059E000ACEBB0E04D915D916D917C91ACECB0E091
:1059F0000D911D912D913C910E94CE351CF011F01E
:105A00000C94042D0C94102DACEBB0E00D911D9175
:105A10002D913C91ACECB0E00D931D932D933C93F4
:105A20000C94A42D023111F00C94262D80912604A3
:105A300081508093260400912604013010F00C94CC
:105A4000242D81E0809326040C94A42D033111F0C1
:105A50000C94662DEAE1F4E00E94FA32E6E2F4E00A
:105A6000A190BB24E2E0F4E0AA0CBB1CAA0CBB1C76
:105A7000EA0DFB1D0E94FF320E946B3418F011F0FA
:105A80000C944A2DE6E0F4E0AAE1B4E00E943F362F
:105A90000C94642DE6E2F4E0A190BB24E2E0F4E093
:105AA000AA0CBB1CAA0CBB1CEA0DFB1D0E94FF32FA
:105AB000EAE1F4E00E94FA320E94F833EDE0F0E00F
:105AC000AAE1B4E00E943F360C94A42D043111F0F9
:105AD0000C94A42DEEE1F4E00E94FA32E6E2F4E048
:105AE000A190BB24E2E0F4E0AA0CBB1CAA0CBB1CF6
:105AF000EA0DFB1D0E94FF320E946B3418F011F07A
:105B00000C948A2DEAE0F4E0AEE1B4E00E943F3666
:105B10000C94A42DE6E2F4E0A190BB24E2E0F4E0D2
:105B2000AA0CBB1CAA0CBB1CEA0DFB1D0E94FF3279
:105B3000EEE1F4E00E94FA320E94F833EDE0F0E08A
:105B4000AEE1B4E00E943F360895EEEEF3E0D1906E
:105B5000E0808FEFE7FE8827F82E082F0E941E3383
:105B60000E945533ECEFF0E70E9459340E94F8335D
:105B7000EDE0F0E0A1EFB3E00E943F36E0EEF3E0AD
:105B80000E94FF32E1EFF3E00E94FA320E94C63336
:105B9000EDE0F0E0A1EFB3E00E943F36A0EEB6E00A
:105BA000AF93BF93E1EFF3E00E94FA320E942C30F2
:105BB00011E001E0BF91AF910E947C35E0EEF6E08C
:105BC000A5EFB3E00E943A36ACECB0E00D911D9128
:105BD0002D913C91A8ECB0E04D915D916D917C913F
:105BE0000E94C935ACE6B0E00D931D932D933D9313
:105BF00041E050E060E070E0A8EDB0E00D911D9153
:105C00002D913C910E94CE3511F00C94822EACE681
:105C1000B0E00D911D912D913C914FE750E060E077
:105C200070E00E94C02FACE6B0E04D935D936D93A1
:105C30007D93ACE6B0E00D911D912D913C91A0E7D4
:105C4000B0E00D931D932D933C93ACE6B0E00D9125
:105C50001D912D913C91AAEEB3E04D915D9157FBC2
:105C60001EF46FEF7FEF02C0662777270E946E3227
:105C7000ACE6B0E00D931D932D933D9300914F0141
:105C8000053011F00C946C2EACECB0E00D911D9130
:105C90002D913C91ACE6B0E04D915D916D917C9180
:105CA0000E94C935ACE6B0E00D931D932D933D9352
:105CB00005EE13E82EE135E0ACE6B0E04D915D91E4
:105CC0006D917C910E94C935ACE6B0E00D931D93B7
:105CD0002D933D930C94802EACE6B0E00D911D9178
:105CE0002D913C91A8ECB0E04D915D916D917C912E
:105CF0000E94C435ACE6B0E00D931D932D933D9307
:105D00000C94112FE8ECF0E00E94FA320E941E334E
:105D1000A1EFB3E00E945033E1EFF3E00E943D3881
:105D2000EDE0F0E0A1EFB3E00E943F36ECECF0E0F4
:105D30000E94FA320E941E33ABE4B1E00E9450335D
:105D4000EBE4F1E00E943D38EDE0F0E0ABE4B1E0DF
:105D50000E943F36E1EFF3E00E94FF32EBE4F1E016
:105D60000E94FA320E94F833EDE0F0E0ABE4B1E0DB
:105D70000E943F36ECEDF0E70E946234EBE4F1E084
:105D80000E94FA320E947033EDE0F0E0ABE4B1E043
:105D90000E943F36EAEEF3E0D190E0808FEFE7FE1D
:105DA0008827F82E082F0E941E330E945533EBE4FB
:105DB000F1E00E94FA320E94C633EDE0F0E0ABE47D
:105DC000B1E00E943F36EBE4F1E00E94FF32E1EFE8
:105DD000F3E00E94FA320E940734EDE0F0E0ABE419
:105DE000B1E00E943F36EBE4F1E00E94FF32ECE9C3
:105DF000F0E70E9459340E94D737EDE0F0E0ABE4C1
:105E0000B1E00E943F36EBE4F1E00E943737EDE06D
:105E1000F0E00E94BC32ACE6B0E0EDE0FF270E946B
:105E20003F36E2E9F0E00E94FA320E941E330E94FF
:105E300055332F933F934F935F93ECE6F0E00E942E
:105E4000FA320E941E335F914F913F912F910E9431
:105E50007033EDE0F0E0ABE4B1E00E943F36A0EE3D
:105E6000B6E0AF93BF93EBE4F1E00E94FA320E94F8
:105E70002C3011E005E0BF91AF910E947C35E0EE3F
:105E8000F6E0A4E3B1E00E943A367091E8007F7D2D
:105E90007093E80008958AE090E00E941D30089514
:105EA000481A590A0895481A8827580A0895ED9102
:105EB000FC91EF5FFF4FFC93EE930895ED91FC9101
:105EC000E150F040FC93EE93089509D00E946432B3
:105ED00000FC10D0089503D01ED001F8F9CF0024A3
:105EE000E89457FF02C009D0689400F80BD010F86E
:105EF0000124089502D009D00895509540954F5F30
:105F00005F4F0895E89417FF0895009510950F5F6F
:105F10001F4F68940895352F242FE894452B11F4D2
:105F200068940895512F402F0027112780E1440FD6
:105F3000551F001F111F021B130B416018F4020FA5
:105F4000131F4E7F8A9599F70895A0EEB6E08D91C4
:105F5000882311F00FD0FBCF08950E945534802D77
:105F600011F008D0FACF089588EE93E066D031970B
:105F7000D9F708950C949031089500FC05D0089548
:105F800030D005D001F8F9CF37D03FD00895842F15
:105F9000952FA62FB72FE894452B462B472B11F4AE
:105FA00068940895402F512F622F732F00271127D7
:105FB00022273327F0E2440F551F661F771F001F6B
:105FC000111F221F331F081B190B2A0B3B0B4160AB
:105FD00028F4080F191F2A1F3B1F4E7FFA9559F707
:105FE00008950024E89477FF02C006D0689400F872
:105FF00009D010F80124089512D04F5F5F4F6F4F02
:106000007F4F0895E89437FF0895009510952095E7
:1060100030950F5F1F4F2F4F3F4F68940895409565
:1060200050956095709508953197F1F708956894AB
:1060300062F80895E89462F80895EF93FF93EE27CD
:10604000E82BE92B31F0E0EDF7E03197F1F701971C
:10605000D1F7FF91EF9108958DE207FD8D938F2D7C
:10606000881F802F881F8F57082F6894F7F8802F7C
:1060700087FF15C080958395082F80E38D938EE26E
:106080008D93802F815228F080E38D9399279C93E4
:10609000089544270A95802F09F196D01FC0805299
:1060A00030F09EE49D9381E48D939D93EFCF442740
:1060B000DF92EF92FF920F938FE1801B11F0082F78
:1060C00083D089D09EE29D930F91FF90EF90DF9057
:1060D00044270395003209F4D7CF2BD03F93E8E64D
:1060E000F1E638E12F2D1E2D0D2DFF24EE24DD24A9
:1060F0004427000F111F221FA8F42F923F920E94E5
:106100005534102C0E945534202C0E945534302CCC
:106110000E9455343197410DD21CE31CF01C3F9076
:106120002F9001C0339631963A9519F73F9107D0D9
:10613000AFCFDD0CEE1CFF1C0A95D9F708950027A0
:1061400019E058D08F93802B11F0039501C08F91E7
:106150001A95B9F7802F882309F496CF8F91805D27
:106160008D930A95D9F792CF0065CD1D80B2E60ECA
:1061700040597307A0ACB90350D6DC01286BEE0080
:1061800094357700CA9A3B0065CD1D00B2E60E003B
:1061900059730700ACB90300D6DC01006BEE0000B8
:1061A000357700009A3B0000CD1D0000E60E000090
:1061B00073070000B9030000DC010000EE000000DE
:1061C000770000003B000000F694E794D7944795D1
:1061D0000A95D1F7089500270DD08F9303958F2D41
:1061E0008E298D29842BC1F78F91805D8D930A951F
:1061F000D9F74CCF1F930F93002710E2440FDD1CFB
:10620000EE1CFF1C001F802F9AE0890B10F0082F56
:1062100043951A9599F7802F0F911F910895442760
:1062200018D0DA98DB9ADD9884E699270E941D3011
:106230009FEF94BBDA9A37D014FCFDCF02D04FEF1A
:1062400008D08FE30FD080EC0DD080E40BD088EB2A
:1062500009C0403420F0D89AD99840540895D99A6A
:10626000D8980895DC9801C0DC9AEF93FF93E6E09C
:10627000F0E00E941430FF91EF9185BBDB98DD9A2E
:10628000000000000000000000000000000000000E
:1062900000000000000000000000000000000000FE
:1062A0000000DD980895DC9804D017FCFCCF089519
:1062B000DC9A992794BB9FEF95BBEF93FF93E6E0A1
:1062C000F0E00E941430FF91EF91DB9ADD9A00001C
:1062D00000000000000000000000000000000000BE
:1062E00000000000000000000000000000000000AE
:1062F00013B2DD9894BB08954427ABDF02D04FEF73
:10630000A8DF00E080E4AEDF88EB800FABDF10E4B5
:106310008827AADF1A95E1F70395083099F70895C1
:10632000EF93FF93509162005F9370906300E09150
:106330006000F09161000E945534202D0E94553478
:10634000302D0E945534002D0E9455348052482F24
:106350000E946636E40FF51F70926300B32E4091E1
:106360006300509162001DD00E945534802D5091E1
:106370006400552309F0809577DF509163005395B1
:1063800050936300BA9459F750916200539550931B
:1063900062002A9509F75F9150936200FF91EF9197
:1063A00008954A955A9555DF88EB850F5BDF80E4A9
:1063B000840F58CF0F921F922F923F920F939F936B
:1063C0004F93052F48E00E947236082E4F91502FB0
:1063D000242E352EE8DF6CDF6BDF422D532DE3DFFB
:1063E000802D0E9465350F91002311F0182A01C0FD
:1063F0001922812D39DF0F913F902F901F900F9020
:106400000895AA24BB24FF24EC81EA80EE1AFF0839
:10641000FB81298033242F1A330881E0EA14FA041F
:106420003CF42FEF3FEFE094F094E80EFA1C02C02A
:1064300021E033272A143A043CF46FEF7FEF2094D5
:106440003094280E3A1C02C061E0772735D02E1414
:106450003F0414F009F017C0CE2CDF2CCC0CDD1C4F
:10646000022C132C000C111C9A81E91761F0E20F29
:10647000A00CB11CAE14BF0424F019F0F60FAC1838
:10648000BD081AD0F1CFC22CD32CCC0CDD1C0E2CA5
:106490001F2C000C111C9981F91711F425960895F1
:1064A000F60FA00CB11CA214B30424F019F0E20FF3
:1064B000AC18BD0801D0EFCF4E2F5F2F98817ACF57
:1064C000480E8827581E08950F92B801469F8001F4
:1064D000479F100D569F100D0F9008950F921F9219
:1064E0002F92C801D901489F80014A9F90014B9F7C
:1064F000202C499F100D211D321D5A9F202C589F82
:10650000100D211D321D599F200D311D689F200D3A
:10651000311D699F300D789F300D2F901F900F9087
:1065200008950E9455340D920020D9F70895369AA7
:106530003699FECF369A3699FECF84B195B108953B
:10654000903041F00D911C91000F111F9A95E1F7C9
:106550001C930E930895903071F00D911D912D9123
:106560003C9136952795179507959A95D1F73C93C9
:106570002E931E930E9308953DD0992711278F2DAA
:10658000880F80E8F82A802F881F08F41FEF41F059
:106590008F57082F07FD04C0003240F08FEF01C075
:1065A0008827982FD82EE82EF82E09C08FE1801B5F
:1065B000082FF694E794D79497950A95D1F711236D
:1065C00051F09095D094E094F09481E0980F882752
:1065D000D81EE81EF81E0F2DFE2CED2CD92E089586
:1065E000D094E094F09491E0D90E9927E91EF91E19
:1065F00010950895D190E190F19001910895219125
:106600003191419151910895102F90E8FF0C001F96
:106610000927990FF7941078652F90E8440F551FBC
:106620005927990F4795607800380895FF0C90E836
:106630009027110F9795F794092F0895102FBD2CCF
:10664000DE2CEF2CF02E11234AF4B094D094E09479
:10665000F0949FEFB91AD90AE90AF90A0EE1FF206E
:1066600039F4FE2CED2CDB2CBB240850C2F76CC097
:1066700032F00A95BB0CDD1CEE1CFF1CF9CF0E940A
:106680004233D4CFB7FE089590E8B91611F4D0FE86
:1066900008959FEFD91AE90AF90A09F403950895B4
:1066A000DD92ED92FD920C930895502F2D2D3E2DED
:1066B0004F2D612F08952DEC3CEC4CEC5DE36627EB
:1066C0000FC098DFF2DFDD24EE2490E8F92E0FE30F
:1066D00007C095DF05C02227332740E251E4662733
:1066E000552351F1002381F18FDF71F116270058F6
:1066F00050580894050B18F407FD03C025C007FD8A
:1067000023C0469537952795F694E794D79422D0E1
:10671000FF202AF0DD0CEE1CFF1C015073F09D2DB4
:10672000969548F0DD203AF4EE202AF491E0D90E57
:106730009927E91EF91E7ACF07C09FE7092FF92A8A
:106740009FEFD92EE92E0895DD24EE24FF240027A3
:10675000112708959F929924AA24BB2488E1D21678
:10676000E306F40628F0D21AE30AF40A089401C0FA
:106770008894991CAA1CBB1CDD0CEE1CFF1C8A957E
:1067800071F7D92CEA2CFB2C9F9008953DDFE1F2A4
:106790005038D1F21627005850580894051F12F4AB
:1067A00018F4CBCF08F0D0CF0BD0FF202AF0BB0CD1
:1067B000DD1CEE1CFF1C3ACF0F5F0BF4BECF36CFB3
:1067C0009F929924AA24BB24992788E1990CAA1C9A
:1067D000BB1CDD1CEE1CFF1C30F4920EA31EB41E6D
:1067E000D91EE91EF91E8A9589F79F90089507DF43
:1067F0000BDF503829F090E869270CC00AF045D02B
:1068000015CF5FE322273327442701C0F8DEFCDEE3
:106810005038B1F3003899F3902F951B8BF312F495
:1068200034D0FACF983118F02227332744279830F4
:1068300028F0232F342F44279850F9CF992329F09B
:106840004695379527959A95D9F7912F962742F037
:1068500014D0B0F6F794E794D7940F5F8BF66DCF12
:1068600010D051F008F4BCDEFF2052F2DD0CEE1C1B
:10687000FF1C0150CBF761CF67CFD20EE31EF41E91
:106880000895D21AE30AF40A0895DF92EF92FF9274
:106890000F931F93D22EE32EF42E052F162F6F91F8
:1068A0005F914F913F912F910895C89531960020A7
:1068B0000895FBDFD02CF9DFE02CF7DFF02CF5DFBB
:1068C000002D0895F2DF202DF0DF302DEEDF402D7A
:1068D000ECDF502D089507FB00680EF40F7757FB8F
:1068E00050680EF45F7707FD02C057FF05C0D2164F
:1068F000E306F406050708952D153E054F055007DC
:1069000008950E941A30E89488278A938A931CDF9E
:1069100011278D918032E9F31197BBD098F08D3219
:1069200029F4109511968C91B4D060F08E3229F430
:1069300011968C91AED008F446C022960E94173072
:1069400081E008958C91A5D0D8F547D01196D0F765
:1069500003958D919ED0E0F38E3229F48C9199D0DD
:1069600010F41196FBCF853419F0853609F055C027
:1069700011968C918ED060F08D3219F08B3221F00F
:10698000DCCF08800094088211968C9182D0A8F602
:106990008053898311968C917CD058F49981990FFA
:1069A000990F0980900D990F8053890F8983873241
:1069B00020F68981988199230AF48195080F2DC0CA
:1069C0008E3289F611968C9164D068F606D018F054
:1069D00011960A95F8CF1196C1CF4F2D3E2D2D2D32
:1069E000DD0CEE1CFF1CA8F0DD0CEE1CFF1C88F07B
:1069F000D20EE31EF41E68F0DD0CEE1CFF1C48F006
:106A0000805309F06894D80E8827E81EF81E08F015
:106A10000895F42EE32ED22E089534D019F116F5F0
:106A2000098308E921D00695882787959F2D9F77B0
:106A3000980FF92E0150000F110F079589818823B7
:106A400079F01AF48195898306C035DE89818A95AB
:106A50008983D9F705C03FDE89818A958983D9F773
:106A60002296089571DEFCCF0DD041F0FF2032F068
:106A70000A9531F0DD0CEE1CFF1CD2F788940895C6
:106A80000894089500240D280E280F28002A0020BD
:106A90000895803320F08A3310F408940895889480
:106AA000089591E005C092E003C094E001C098E031
:106AB000FCDE0D929A95E1F7089582E001C084E032
:106AC00099279D938A95E9F7089591E0882321F00D
:106AD0008894991F8A95E9F7892F909508959927A9
:106AE0008D9193958823E1F7939511968C93119747
:106AF0008E919A95D1F70895EA2FFB2F00244C919F
:106B00008D9103948E32E1F711248D911394882393
:106B1000E1F71A94101640F41197202F21192395AC
:106B200080E38D932A95E9F7113039F59927AE2F37
:106B3000BF2FA00DB91FA00FB91F8C919C93853357
:106B400008F421C031E08E918E32E9F38D3241F0AC
:106B5000830F8A3319F480E331E001C033278C932B
:106B6000AE1789F7332341F0AE2FBF2FB8DF81E393
:106B70004D3209F43196808308958827E00DF81F7F
:106B8000E00FF81F80830895040F151F261F371F7D
:106B90000895041B150B260B370B089504171507D2
:106BA000260737070895000F111F221F331F08956E
:106BB00000951095209530950F5F1F4F2F4F3F4F39
:106BC0000895019110810EC00191119121913081A0
:106BD0000BC00191108117FF05C03FEF2FEF04C0DC
:106BE000008111272227332737FF03C0E1DF8DE221
:106BF0008D93CF93DF93CF92DF92EF92AA24BB24A1
:106C0000CC24DD24EE2440E2CAE0DD2755E093E306
:106C10008881890F87FD9F7083FD907F891B8993F1
:106C20005A95A9F7C0DFAA1CBB1CCC1CDD1CEE1CAE
:106C30004A9551F7E894EFE0FF2782910ED0EB30B0
:106C4000E0F71EF068948A2D0CD088278D93EF9082
:106C5000DF90CF90DF91CF910895982F829501D04A
:106C6000892F8F70805D26F0803309F40895689431
:106C70008D93089581918D938823E1F7089594E091
:106C800081918D939A95E1F70895E199FECFEEBB3E
:106C9000FFBB3196089591E001C092E07B3751F43B
:106CA0007FB7F894F2DF8D918DBBE29AE19A9A95C5
:106CB000C9F77FBF7727089591E001C092E0E5DF33
:106CC000E09A8DB38D939A95D1F70895FF93552748
:106CD000F8E0469508F4500F57954795FA95D1F787
:106CE000FF910895FF93881BF9E0001FFA9511F4B6
:106CF000FF910895881F841B18F4840F8894F5CFA2
:106D00000894F3CF002711272D913D910217130707
:106D100010F4022F132F3197B9F708950FEF1FEFDB
:106D20002D913D910217130710F0022F132F319769
:106D3000B9F708950FEF1FEF8827992744275527A4
:106D40002D913D9101960217130720F0022F132F6A
:106D5000482F592F3197A1F7089588E00FB6F8947E
:106D60005A924A92E42DF52DA42DB52D480E882770
:106D7000581E0FBE08950FB6F894499059900FBE53
:106D8000089538DC41DC0395AAF087E1DD0CEE1CA8
:106D9000FF1C8A9589F00A95CAF7FF205AF0002453
:106DA0000D280E280F28002039F00A95DD0CEE1C66
:106DB000FF1CDAF70A953ACCC7CCC6CC1BDC002303
:106DC000E2F360DE19F4B9DC0068089585E0C6DFFF
:106DD000FF0C001F04830FE70695F79456D1506807
:106DE00016DD5EDC139721E438E743ED5BEBCEDC88
:106DF00027E831ED43E15DE3D6D02EE03CE343EC00
:106E00005DEBD1D022E83DEA4BE25EE3CCD02CEE44
:106E100032E846E75EEBC7D020E931EE49EA5EE3AF
:106E2000C2D020E83FEE4FEF5EEBBDD024EC3FEF49
:106E30004FE75FE3B8D034DC139784818F5799F024
:106E40002AF4D82E0FEFE02EF02E04C0D82EEE2418
:106E5000FF240027F3DB28E132E741E35FE396DC20
:106E6000CEDB3497D4DC87CFC5DB80E003C0C2DB48
:106E7000802F8078882321F0DF92EF92FF920F938A
:106E80008F93C2DB802F839512F45EDC1BC080954C
:106E90008A95885E0AF415C088501AF40CD0D9225D
:106EA00010C0DD2488501AF406D0E9220AC0EE246E
:106EB00002D0F92206C09FEF8770990F8A95EAF7F2
:106EC0000895B4DB8F918823D9F35F914F913F915F
:106ED0002F910F9300DD0F9199F390F3D6D0506866
:106EE00096CC2BDC48CF86DB86E038DF05830F7736
:106EF0002BE33AEA48EB5FE349DCD2DB139741D05E
:106F000028F4858188236AF71FDC35CF8F77848347
:106F100071DB349737DFC4DB139723E632E446E3B3
:106F200057EB34DC29ED37EA4AE159E33CD026E55A
:106F300038E14EEA5AEB37D026E53CE84DE15CE318
:106F400032D02DEC37E543E65DEB2DD02DEE3DEF55
:106F500045E75EE328D028E132E741E35FEB23D049
:106F600094D055DCA2DBDD24EE24FF2404818FE7DE
:106F7000080F0695F794B4DB8581881F08F4A2DB1F
:106F8000FACE42DB8827039512F4889408950730DF
:106F90001AF0812F08940895FF1C881F0A95E2F7C4
:106FA000812B8894089533DC2ADB3497EFCB0F9341
:106FB000FF92EF92EDB7FEB7DF925F934F933F934F
:106FC000ADB7BEB72F9306D0EDB7FEB73896EDBF7D
:106FD000FEBF089588278A93FA93EA93BA93AA93F7
:106FE0000E94FA32EA2FFB2F0E94FF320E940433E4
:106FF000503819F40038B1F13BC0003819F457FD8E
:107000002CC02DC00F3771F15F3761F117FF11C030
:10701000E881F9810E94BC328827D0FA87F98C83F5
:107020000E941E33E881F9810E94FF320E946B3476
:10703000C9F4EA81FB810E94FA320F770E94DF36A1
:10704000E881F9810E94FF320E94C6330E947437A2
:107050008C8187FB07F9259608950FE701C000276B
:10706000882702C00FE78FEFF82EE82ED82EF3CF37
:107070000FE380E8F82E8827F8CFBCDAA0DE29EDF0
:107080003BE54EED5EE30C94C6335FE340E8332707
:1070900022270895CDCCCC3D0000803F0000204148
:1070A0000000C84200007A440AD7234A01000000C9
:1070B0000000A04082E2473E0000004400005C4225
:1070C00000006442000000BF000080BF0000A0413B
:1070D0007AE51D42BD378635002474490000FE4222
:1070E000CDCCC7429AF979449A3F1C4600401C46D1
:1070F000F34FC34702000000804FC3470000E04049
:10710000203130487A00313030487A0020316B48E5
:107110007A0031306B487A00203130306B002031FA
:107120004D487A0020202020204E412D3031202053
:107130002020202000006369726375697420616EED
:10714000616C797A65720000202020207665722EAD
:1071500020322E35202020200000206D6164652023
:107160006279207370366672652000002D2D2D2DFA
:107170002D2D2D2D2D2D2D2D2D2D2D2D0000687417
:1071800074703A2F2F6C782D6E65742E706C000021
:107190004F4B0000497A6D2E207720716F6C6F6322
:1071A0006500497A6D6570656E69652020646F625F
:1071B000702E0000497A6D2E206D6F5B6E6F6374C8
:1071C00069004B4342206D6F637420200000416EC4
:1071D000616C697A206371656B74706100004B614A
:1071E0006C6962706F776B6100004B616C696270F3
:1071F0006F776B61204B43420000426F7A6270618F
:107200007400436C65642E20796B617A616E694A03
:107210006D3A0000312E4F74636F65642E207778CD
:107220006F6420200000322E48617B6D69742E202F
:10723000454E544552200000425C716F6C6E75746F
:10724000202020202020202000006B616C696270CB
:107250002E206D6F5B6E6F632E3F0000497A6D6567
:1072600070656E69652020202020202000004B6181
:107270006C6962706F776B612020202020200000F5
:10728000312E4F746B6C795D6974206F74202020EF
:1072900000007563746F5D6E2E206D6F5B6E6F63A3
:1072A00074750000312E486F646B6C755D697420D5
:1072B0006B2020200000322E4963716F6C2E203C21
:1072C0002D2069202D3E00007963742E2079706F87
:1072D00077656E60206D42740000332E5A617765C9
:1072E000702F2E20454E54455220000059706F7764
:1072F0002E206D42743D20002020202020202020C0
:1073000020202020202020200000202020202020BD
:1073100020202020000075572000572000006D57C6
:10732000200064426D004963716F6C7A2E204B43DC
:1073300042206D6F63740000312E486F646B6C2EB9
:1073400020776E652F6E696A000020206D6F637470
:10735000206B204E4130312020200000322E497A0F
:107360006D6570656E696520632020200000202017
:10737000776E652F6E756D206D6F63746F6D000095
:10738000332E486F646B6C7D5D697465206B2020C3
:10739000000020206D6F637479203530206F6D20E0
:1073A00020200000342E48617B6D69742E20454EEC
:1073B0005445522000004963716F6C7A2E20646F2F
:1073C000716F6C6E2E3A0000312E4F64636F6564EE
:1073D0002E206B6F6D712E2000002020697A2070A6
:1073E000617A666D6120202020200000312E436FDD
:1073F0006564656E6974652077786F64000020208D
:107400006320775C786F646F6D202020202000005F
:10741000312E204F646B6C7D5D697420202020200C
:10742000000020697A206D6F637461203530206F11
:107430006D200000322E48617B6D69742E20454E10
:1074400054455220222000004B616C6962702E204E
:107450006364656C616E61200000516F646B6C2E1B
:1074600020772070617A666D202000006B6F6D714F
:107470002E20646C4A2071706F772E2000004D49D9
:107480004E203D2000004D4158203D200000447911
:107490006E203D200000206442004D200000644228
:1074A0000000494E46002020202020202053575223
:1074B0003D004D696E3D0000496E643D000046721E
:1074C0003D004D487A00513D00004C783D00754824
:1074D000000043783D00704600004D00497A6D651C
:1074E00070656E696500537465703A202020202015
:1074F0002000537461723A202000537461723A2064
:10750000000053746F703A20200053746F703A205B
:1075100000004C494E004C4F4700537765703A20AD
:107520002020202020202000532F530044454C00D1
:107530004D6F64653A2020202020202020004465E3
:107540006C743A20200044656C743A2000004C436F
:1075500073743A2020202020202020302E3100007B
:107560004C4373743A2020202020202020202031FA
:1075700000004C4373743A2020202020202020203B
:10758000313000004C4373743A202020202020200A
:107590002031303000004C4373743A2020202020EA
:1075A00020203130303000004C7220203A20202042
:1075B000202020004C7220203A2020202020000093
:1075C0004C7220203A20202020004C7220203A20AB
:1075D000202000004C7220203A20200043722020FE
:1075E0003A20202020202000437220203A20202012
:1075F00020200000437220203A20202020004372E7
:1076000020203A2020200000437220203A20200031
:0A76100053415645202020202000A1
:00000001FF
